 suspendthrd003

 Timestamp is 55b2d268 (reproducible build file hash)

 Preferred load address is 0000000180000000

 Start         Length     Name                   Class
 0001:00000000 00003c30H .text$mn                CODE
 0001:00003c30 00000036H .text$mn$00             CODE
 0001:00003c66 00000092H .text$x                 CODE
 0002:00000000 000001d0H .idata$5                DATA
 0002:000001d0 00000038H .00cfg                  DATA
 0002:00000208 00000008H .CRT$XCA                DATA
 0002:00000210 00000008H .CRT$XCZ                DATA
 0002:00000218 00000008H .CRT$XIA                DATA
 0002:00000220 00000008H .CRT$XIC                DATA
 0002:00000228 00000008H .CRT$XIZ                DATA
 0002:00000230 00000008H .CRT$XLA                DATA
 0002:00000238 00000008H .CRT$XLZ                DATA
 0002:00000240 00000008H .CRT$XPA                DATA
 0002:00000248 00000008H .CRT$XPZ                DATA
 0002:00000250 00000008H .CRT$XTA                DATA
 0002:00000258 00000008H .CRT$XTZ                DATA
 0002:00000260 00000000H .gehcont$y              DATA
 0002:00000260 00000000H .gfids$y                DATA
 0002:00000260 000022a0H .rdata                  DATA
 0002:00002500 00000000H .rdata$CastGuardVftablesA DATA
 0002:00002500 00000000H .rdata$CastGuardVftablesC DATA
 0002:00002500 00000028H .rdata$T                DATA
 0002:00002528 000000bcH .rdata$voltmd           DATA
 0002:000025e4 0000031cH .rdata$zzzdbg           DATA
 0002:00002900 00000008H .rtc$IAA                DATA
 0002:00002908 00000008H .rtc$IZZ                DATA
 0002:00002910 00000008H .rtc$TAA                DATA
 0002:00002918 00000008H .rtc$TZZ                DATA
 0002:00002920 00000004H .tls                    DATA
 0002:00002924 00000004H .tls$                   DATA
 0002:00002928 00000008H .tls$ZZZ                DATA
 0002:00002930 00000340H .xdata                  DATA
 0002:00002c70 00000368H .edata                  DATA
 0002:00002fd8 0000008cH .idata$2                DATA
 0002:00003064 00000014H .idata$3                DATA
 0002:00003078 000001d0H .idata$4                DATA
 0002:00003248 00000490H .idata$6                DATA
 0003:00000000 00000080H .data                   DATA
 0003:00000080 0001b368H .bss                    DATA
 0004:00000000 000003d8H .pdata                  DATA

  Address         Publics by Value              Rva+Base               Lib:Object

 0000:00000000       __AbsoluteZero             0000000000000000     <absolute>
 0000:00000000       ___safe_se_handler_count   0000000000000000     <absolute>
 0000:00000000       ___safe_se_handler_table   0000000000000000     <absolute>
 0000:00000000       __arm64x_extra_rfe_table   0000000000000000     <absolute>
 0000:00000000       __arm64x_extra_rfe_table_size 0000000000000000     <absolute>
 0000:00000000       __arm64x_native_entrypoint 0000000000000000     <absolute>
 0000:00000000       __arm64x_redirection_metadata 0000000000000000     <absolute>
 0000:00000000       __arm64x_redirection_metadata_count 0000000000000000     <absolute>
 0000:00000000       __dynamic_value_reloc_table 0000000000000000     <absolute>
 0000:00000000       __enclave_config           0000000000000000     <absolute>
 0000:00000000       __guard_check_icall_a64n_fptr 0000000000000000     <absolute>
 0000:00000000       __guard_eh_cont_count      0000000000000000     <absolute>
 0000:00000000       __guard_eh_cont_table      0000000000000000     <absolute>
 0000:00000000       __guard_fids_count         0000000000000000     <absolute>
 0000:00000000       __guard_fids_table         0000000000000000     <absolute>
 0000:00000000       __guard_iat_count          0000000000000000     <absolute>
 0000:00000000       __guard_iat_table          0000000000000000     <absolute>
 0000:00000000       __guard_longjmp_count      0000000000000000     <absolute>
 0000:00000000       __guard_longjmp_table      0000000000000000     <absolute>
 0000:00000000       __hybrid_auxiliary_iat     0000000000000000     <absolute>
 0000:00000000       __hybrid_auxiliary_iat_copy 0000000000000000     <absolute>
 0000:00000000       __hybrid_code_map          0000000000000000     <absolute>
 0000:00000000       __hybrid_code_map_count    0000000000000000     <absolute>
 0000:00000000       __x64_code_ranges_to_entry_points 0000000000000000     <absolute>
 0000:00000000       __x64_code_ranges_to_entry_points_count 0000000000000000     <absolute>
 0000:00000100       __guard_flags              0000000000000100     <absolute>
 0000:00000000       __ImageBase                0000000180000000     <linker-defined>
 0001:00000000       ?NewObject@JNIEnv_@@QEAAPEAV_jobject@@PEAV_jclass@@PEAU_jmethodID@@ZZ 0000000180001000 f i libsuspendthrd003.obj
 0001:00000028       ?TranslateError@@YAPEBDW4jvmtiError@@@Z 0000000180001028 f   libsuspendthrd003.obj
 0001:000002e0       ?TranslateState@@YAPEBDH@Z 00000001800012e0 f   libsuspendthrd003.obj
 0001:00000424       ?nsk_jni_check_exception@@YAHPEAUJNIEnv_@@QEBDH@Z 0000000180001424 f   libsuspendthrd003.obj
 0001:00000568       ?nsk_jni_lverify@@YAHHPEAUJNIEnv_@@HQEBDH1ZZ 0000000180001568 f   libsuspendthrd003.obj
 0001:00000608       Agent_Initialize           0000000180001608 f   libsuspendthrd003.obj
 0001:000007e4       Agent_OnAttach             00000001800017e4 f   libsuspendthrd003.obj
 0001:000007e4       Agent_OnLoad               00000001800017e4 f   libsuspendthrd003.obj
 0001:000007ec       Java_nsk_jvmti_unit_FollowReferences_FollowRefObjects_addRefToVerify 00000001800017ec f   libsuspendthrd003.obj
 0001:000009c4       Java_nsk_jvmti_unit_FollowReferences_FollowRefObjects_getTag 00000001800019c4 f   libsuspendthrd003.obj
 0001:00000a84       Java_nsk_jvmti_unit_FollowReferences_FollowRefObjects_resetRefsToVerify 0000000180001a84 f   libsuspendthrd003.obj
 0001:00000a8c       Java_nsk_jvmti_unit_FollowReferences_FollowRefObjects_resetTags 0000000180001a8c f   libsuspendthrd003.obj
 0001:00000ad0       Java_nsk_jvmti_unit_FollowReferences_FollowRefObjects_setTag 0000000180001ad0 f   libsuspendthrd003.obj
 0001:00000d28       Java_nsk_share_jvmti_ArgumentHandler_getAgentOptionsString 0000000180001d28 f   libsuspendthrd003.obj
 0001:00000dd8       Java_nsk_share_jvmti_DebugeeClass_checkStatus 0000000180001dd8 f   libsuspendthrd003.obj
 0001:00000e60       Java_nsk_share_jvmti_DebugeeClass_resetAgentData 0000000180001e60 f   libsuspendthrd003.obj
 0001:00000ec0       Java_nsk_share_jvmti_RedefineAgent_agentStatus 0000000180001ec0 f   libsuspendthrd003.obj
 0001:00000ecc       Java_nsk_share_jvmti_RedefineAgent_isRedefined 0000000180001ecc f   libsuspendthrd003.obj
 0001:00000ed8       Java_nsk_share_jvmti_RedefineAgent_redefineAttempted 0000000180001ed8 f   libsuspendthrd003.obj
 0001:00000ee4       MA_checkStatus             0000000180001ee4 f   libsuspendthrd003.obj
 0001:00000f88       __local_stdio_printf_options 0000000180001f88 f i libsuspendthrd003.obj
 0001:000018bc       exitOnError                00000001800028bc f   libsuspendthrd003.obj
 0001:00001970       fprintf                    0000000180002970 f i libsuspendthrd003.obj
 0001:000019b4       nsk_complain               00000001800029b4 f   libsuspendthrd003.obj
 0001:000019e0       nsk_jvmti_createJVMTIEnv   00000001800029e0 f   libsuspendthrd003.obj
 0001:00001b10       nsk_jvmti_lverify          0000000180002b10 f   libsuspendthrd003.obj
 0001:00001c00       nsk_jvmti_parseOptions     0000000180002c00 f   libsuspendthrd003.obj
 0001:00001e50       nsk_jvmti_resetAgentData   0000000180002e50 f   libsuspendthrd003.obj
 0001:00001ed0       nsk_jvmti_resumeSync       0000000180002ed0 f   libsuspendthrd003.obj
 0001:00001f78       nsk_jvmti_setFailStatus    0000000180002f78 f   libsuspendthrd003.obj
 0001:00001fb4       nsk_jvmti_threadByName     0000000180002fb4 f   libsuspendthrd003.obj
 0001:000022d4       nsk_jvmti_waitForSync      00000001800032d4 f   libsuspendthrd003.obj
 0001:000023d8       nsk_lcomplain              00000001800033d8 f   libsuspendthrd003.obj
 0001:000023f8       nsk_ldisplay               00000001800033f8 f   libsuspendthrd003.obj
 0001:00002418       nsk_ltrace                 0000000180003418 f   libsuspendthrd003.obj
 0001:00002438       nsk_lvcomplain             0000000180003438 f   libsuspendthrd003.obj
 0001:000025f0       nsk_lvdisplay              00000001800035f0 f   libsuspendthrd003.obj
 0001:0000263c       nsk_lverify                000000018000363c f   libsuspendthrd003.obj
 0001:00002698       nsk_lvtrace                0000000180003698 f   libsuspendthrd003.obj
 0001:000026f8       nsk_printf                 00000001800036f8 f   libsuspendthrd003.obj
 0001:00002720       nsk_vprintf                0000000180003720 f   libsuspendthrd003.obj
 0001:000027d4       printf                     00000001800037d4 f i libsuspendthrd003.obj
 0001:00002cfc       __raise_securityfailure    0000000180003cfc f   MSVCRT:gs_report.obj
 0001:00002d30       __report_gsfailure         0000000180003d30 f   MSVCRT:gs_report.obj
 0001:00002f70       __GSHandlerCheck           0000000180003f70 f   MSVCRT:gshandler.obj
 0001:00002f90       __GSHandlerCheckCommon     0000000180003f90 f   MSVCRT:gshandler.obj
 0001:00003000       __security_check_cookie    0000000180004000 f   MSVCRT:amdsecgs.obj
 0001:00003340       _DllMainCRTStartup         0000000180004340 f   MSVCRT:dll_dllmain.obj
 0001:00003380       __scrt_acquire_startup_lock 0000000180004380 f   MSVCRT:utility.obj
 0001:000033bc       __scrt_dllmain_after_initialize_c 00000001800043bc f   MSVCRT:utility.obj
 0001:000033f0       __scrt_dllmain_before_initialize_c 00000001800043f0 f   MSVCRT:utility.obj
 0001:00003408       __scrt_dllmain_crt_thread_attach 0000000180004408 f   MSVCRT:utility.obj
 0001:00003430       __scrt_dllmain_crt_thread_detach 0000000180004430 f   MSVCRT:utility.obj
 0001:00003448       __scrt_dllmain_exception_filter 0000000180004448 f   MSVCRT:utility.obj
 0001:000034a8       __scrt_dllmain_uninitialize_c 00000001800044a8 f   MSVCRT:utility.obj
 0001:000034d8       __scrt_dllmain_uninitialize_critical 00000001800044d8 f   MSVCRT:utility.obj
 0001:000034ec       __scrt_initialize_crt      00000001800044ec f   MSVCRT:utility.obj
 0001:00003538       __scrt_initialize_onexit_tables 0000000180004538 f   MSVCRT:utility.obj
 0001:000035c4       __scrt_is_nonwritable_in_current_image 00000001800045c4 f   MSVCRT:utility.obj
 0001:0000365c       __scrt_release_startup_lock 000000018000465c f   MSVCRT:utility.obj
 0001:00003680       __scrt_uninitialize_crt    0000000180004680 f   MSVCRT:utility.obj
 0001:000036ac       _onexit                    00000001800046ac f   MSVCRT:utility.obj
 0001:000036e8       atexit                     00000001800046e8 f   MSVCRT:utility.obj
 0001:00003700       __crt_debugger_hook        0000000180004700 f   MSVCRT:utility_desktop.obj
 0001:00003708       __scrt_fastfail            0000000180004708 f   MSVCRT:utility_desktop.obj
 0001:00003854       _guard_check_icall_nop     0000000180004854 f i MSVCRT:guard_support.obj
 0001:00003858       __security_init_cookie     0000000180004858 f   MSVCRT:gs_support.obj
 0001:00003904       DllMain                    0000000180004904 f   MSVCRT:dll_dllmain_stub.obj
 0001:00003928       ?__scrt_initialize_type_info@@YAXXZ 0000000180004928 f   MSVCRT:tncleanup.obj
 0001:00003938       ?__scrt_uninitialize_type_info@@YAXXZ 0000000180004938 f   MSVCRT:tncleanup.obj
 0001:00003944       __local_stdio_scanf_options 0000000180004944 f i MSVCRT:default_local_stdio_options.obj
 0001:0000394c       __scrt_initialize_default_local_stdio_options 000000018000494c f   MSVCRT:default_local_stdio_options.obj
 0001:00003968       __scrt_get_dyn_tls_init_callback 0000000180004968 f   MSVCRT:dyn_tls_init.obj
 0001:00003970       _RTC_Initialize            0000000180004970 f   MSVCRT:initsect.obj
 0001:000039ac       _RTC_Terminate             00000001800049ac f   MSVCRT:initsect.obj
 0001:000039e8       __isa_available_init       00000001800049e8 f   MSVCRT:cpu_disp.obj
 0001:00003b94       _get_startup_argv_mode     0000000180004b94 f   MSVCRT:argv_mode.obj
 0001:00003b9c       __scrt_is_ucrt_dll_in_use  0000000180004b9c f   MSVCRT:ucrt_detection.obj
 0001:00003bb0       memcpy                     0000000180004bb0 f   vcruntime:VCRUNTIME140.dll
 0001:00003bb6       memset                     0000000180004bb6 f   vcruntime:VCRUNTIME140.dll
 0001:00003bbc       strchr                     0000000180004bbc f   vcruntime:VCRUNTIME140.dll
 0001:00003bc2       __C_specific_handler       0000000180004bc2 f   vcruntime:VCRUNTIME140.dll
 0001:00003bc8       __std_type_info_destroy_list 0000000180004bc8 f   vcruntime:VCRUNTIME140.dll
 0001:00003bce       strcat                     0000000180004bce f   ucrt:api-ms-win-crt-string-l1-1-0.dll
 0001:00003bd4       strcmp                     0000000180004bd4 f   ucrt:api-ms-win-crt-string-l1-1-0.dll
 0001:00003bda       strlen                     0000000180004bda f   ucrt:api-ms-win-crt-string-l1-1-0.dll
 0001:00003be0       _initterm                  0000000180004be0 f   ucrt:api-ms-win-crt-runtime-l1-1-0.dll
 0001:00003be6       _initterm_e                0000000180004be6 f   ucrt:api-ms-win-crt-runtime-l1-1-0.dll
 0001:00003bec       _seh_filter_dll            0000000180004bec f   ucrt:api-ms-win-crt-runtime-l1-1-0.dll
 0001:00003bf2       _configure_narrow_argv     0000000180004bf2 f   ucrt:api-ms-win-crt-runtime-l1-1-0.dll
 0001:00003bf8       _initialize_narrow_environment 0000000180004bf8 f   ucrt:api-ms-win-crt-runtime-l1-1-0.dll
 0001:00003bfe       _initialize_onexit_table   0000000180004bfe f   ucrt:api-ms-win-crt-runtime-l1-1-0.dll
 0001:00003c04       _register_onexit_function  0000000180004c04 f   ucrt:api-ms-win-crt-runtime-l1-1-0.dll
 0001:00003c0a       _execute_onexit_table      0000000180004c0a f   ucrt:api-ms-win-crt-runtime-l1-1-0.dll
 0001:00003c10       _crt_atexit                0000000180004c10 f   ucrt:api-ms-win-crt-runtime-l1-1-0.dll
 0001:00003c16       _cexit                     0000000180004c16 f   ucrt:api-ms-win-crt-runtime-l1-1-0.dll
 0001:00003c1c       __acrt_initialize          0000000180004c1c f   MSVCRT:ucrt_stubs.obj
 0001:00003c1c       __acrt_thread_attach       0000000180004c1c f   MSVCRT:ucrt_stubs.obj
 0001:00003c1c       __acrt_thread_detach       0000000180004c1c f   MSVCRT:ucrt_stubs.obj
 0001:00003c1c       __acrt_uninitialize        0000000180004c1c f   MSVCRT:ucrt_stubs.obj
 0001:00003c1c       __acrt_uninitialize_critical 0000000180004c1c f   MSVCRT:ucrt_stubs.obj
 0001:00003c1c       __scrt_stub_for_acrt_initialize 0000000180004c1c f   MSVCRT:ucrt_stubs.obj
 0001:00003c1c       __scrt_stub_for_acrt_thread_attach 0000000180004c1c f   MSVCRT:ucrt_stubs.obj
 0001:00003c1c       __scrt_stub_for_acrt_thread_detach 0000000180004c1c f   MSVCRT:ucrt_stubs.obj
 0001:00003c1c       __scrt_stub_for_acrt_uninitialize 0000000180004c1c f   MSVCRT:ucrt_stubs.obj
 0001:00003c1c       __scrt_stub_for_acrt_uninitialize_critical 0000000180004c1c f   MSVCRT:ucrt_stubs.obj
 0001:00003c1c       __vcrt_initialize          0000000180004c1c f   MSVCRT:ucrt_stubs.obj
 0001:00003c1c       __vcrt_thread_attach       0000000180004c1c f   MSVCRT:ucrt_stubs.obj
 0001:00003c1c       __vcrt_thread_detach       0000000180004c1c f   MSVCRT:ucrt_stubs.obj
 0001:00003c1c       __vcrt_uninitialize        0000000180004c1c f   MSVCRT:ucrt_stubs.obj
 0001:00003c1c       __vcrt_uninitialize_critical 0000000180004c1c f   MSVCRT:ucrt_stubs.obj
 0001:00003c20       __scrt_stub_for_is_c_termination_complete 0000000180004c20 f   MSVCRT:ucrt_stubs.obj
 0001:00003c20       _is_c_termination_complete 0000000180004c20 f   MSVCRT:ucrt_stubs.obj
 0001:00003c40       _guard_dispatch_icall_nop  0000000180004c40 f   MSVCRT:guard_dispatch.obj
 0001:00003c60       _guard_xfg_dispatch_icall_nop 0000000180004c60 f   MSVCRT:guard_xfg_dispatch.obj
 0002:00000000       __imp_RtlCaptureContext    0000000180005000     kernel32:KERNEL32.dll
 0002:00000008       __imp_RtlLookupFunctionEntry 0000000180005008     kernel32:KERNEL32.dll
 0002:00000010       __imp_RtlVirtualUnwind     0000000180005010     kernel32:KERNEL32.dll
 0002:00000018       __imp_UnhandledExceptionFilter 0000000180005018     kernel32:KERNEL32.dll
 0002:00000020       __imp_SetUnhandledExceptionFilter 0000000180005020     kernel32:KERNEL32.dll
 0002:00000028       __imp_GetCurrentProcess    0000000180005028     kernel32:KERNEL32.dll
 0002:00000030       __imp_TerminateProcess     0000000180005030     kernel32:KERNEL32.dll
 0002:00000038       __imp_IsProcessorFeaturePresent 0000000180005038     kernel32:KERNEL32.dll
 0002:00000040       __imp_CloseHandle          0000000180005040     kernel32:KERNEL32.dll
 0002:00000048       __imp_InitializeCriticalSectionAndSpinCount 0000000180005048     kernel32:KERNEL32.dll
 0002:00000050       __imp_DeleteCriticalSection 0000000180005050     kernel32:KERNEL32.dll
 0002:00000058       __imp_CreateEventW         0000000180005058     kernel32:KERNEL32.dll
 0002:00000060       __imp_GetModuleHandleW     0000000180005060     kernel32:KERNEL32.dll
 0002:00000068       __imp_GetProcAddress       0000000180005068     kernel32:KERNEL32.dll
 0002:00000070       __imp_IsDebuggerPresent    0000000180005070     kernel32:KERNEL32.dll
 0002:00000078       __imp_QueryPerformanceCounter 0000000180005078     kernel32:KERNEL32.dll
 0002:00000080       __imp_GetCurrentProcessId  0000000180005080     kernel32:KERNEL32.dll
 0002:00000088       __imp_GetCurrentThreadId   0000000180005088     kernel32:KERNEL32.dll
 0002:00000090       __imp_GetSystemTimeAsFileTime 0000000180005090     kernel32:KERNEL32.dll
 0002:00000098       __imp_DisableThreadLibraryCalls 0000000180005098     kernel32:KERNEL32.dll
 0002:000000a0       __imp_InitializeSListHead  00000001800050a0     kernel32:KERNEL32.dll
 0002:000000a8       \177KERNEL32_NULL_THUNK_DATA 00000001800050a8     kernel32:KERNEL32.dll
 0002:000000b0       __imp_memcpy               00000001800050b0     vcruntime:VCRUNTIME140.dll
 0002:000000b8       __imp_memset               00000001800050b8     vcruntime:VCRUNTIME140.dll
 0002:000000c0       __imp_strchr               00000001800050c0     vcruntime:VCRUNTIME140.dll
 0002:000000c8       __imp___C_specific_handler 00000001800050c8     vcruntime:VCRUNTIME140.dll
 0002:000000d0       __imp___std_type_info_destroy_list 00000001800050d0     vcruntime:VCRUNTIME140.dll
 0002:000000d8       \177VCRUNTIME140_NULL_THUNK_DATA 00000001800050d8     vcruntime:VCRUNTIME140.dll
 0002:000000e0       __imp_strtol               00000001800050e0     ucrt:api-ms-win-crt-convert-l1-1-0.dll
 0002:000000e8       \177api-ms-win-crt-convert-l1-1-0_NULL_THUNK_DATA 00000001800050e8     ucrt:api-ms-win-crt-convert-l1-1-0.dll
 0002:000000f0       __imp_malloc               00000001800050f0     ucrt:api-ms-win-crt-heap-l1-1-0.dll
 0002:000000f8       __imp_free                 00000001800050f8     ucrt:api-ms-win-crt-heap-l1-1-0.dll
 0002:00000100       \177api-ms-win-crt-heap-l1-1-0_NULL_THUNK_DATA 0000000180005100     ucrt:api-ms-win-crt-heap-l1-1-0.dll
 0002:00000108       __imp__errno               0000000180005108     ucrt:api-ms-win-crt-runtime-l1-1-0.dll
 0002:00000110       __imp_exit                 0000000180005110     ucrt:api-ms-win-crt-runtime-l1-1-0.dll
 0002:00000118       __imp__cexit               0000000180005118     ucrt:api-ms-win-crt-runtime-l1-1-0.dll
 0002:00000120       __imp__crt_atexit          0000000180005120     ucrt:api-ms-win-crt-runtime-l1-1-0.dll
 0002:00000128       __imp__execute_onexit_table 0000000180005128     ucrt:api-ms-win-crt-runtime-l1-1-0.dll
 0002:00000130       __imp__register_onexit_function 0000000180005130     ucrt:api-ms-win-crt-runtime-l1-1-0.dll
 0002:00000138       __imp__initialize_onexit_table 0000000180005138     ucrt:api-ms-win-crt-runtime-l1-1-0.dll
 0002:00000140       __imp__initialize_narrow_environment 0000000180005140     ucrt:api-ms-win-crt-runtime-l1-1-0.dll
 0002:00000148       __imp__configure_narrow_argv 0000000180005148     ucrt:api-ms-win-crt-runtime-l1-1-0.dll
 0002:00000150       __imp__seh_filter_dll      0000000180005150     ucrt:api-ms-win-crt-runtime-l1-1-0.dll
 0002:00000158       __imp__initterm_e          0000000180005158     ucrt:api-ms-win-crt-runtime-l1-1-0.dll
 0002:00000160       __imp__initterm            0000000180005160     ucrt:api-ms-win-crt-runtime-l1-1-0.dll
 0002:00000168       \177api-ms-win-crt-runtime-l1-1-0_NULL_THUNK_DATA 0000000180005168     ucrt:api-ms-win-crt-runtime-l1-1-0.dll
 0002:00000170       __imp___acrt_iob_func      0000000180005170     ucrt:api-ms-win-crt-stdio-l1-1-0.dll
 0002:00000178       __imp_fflush               0000000180005178     ucrt:api-ms-win-crt-stdio-l1-1-0.dll
 0002:00000180       __imp___stdio_common_vsprintf 0000000180005180     ucrt:api-ms-win-crt-stdio-l1-1-0.dll
 0002:00000188       __imp___stdio_common_vfprintf 0000000180005188     ucrt:api-ms-win-crt-stdio-l1-1-0.dll
 0002:00000190       \177api-ms-win-crt-stdio-l1-1-0_NULL_THUNK_DATA 0000000180005190     ucrt:api-ms-win-crt-stdio-l1-1-0.dll
 0002:00000198       __imp_strcat               0000000180005198     ucrt:api-ms-win-crt-string-l1-1-0.dll
 0002:000001a0       __imp_strcmp               00000001800051a0     ucrt:api-ms-win-crt-string-l1-1-0.dll
 0002:000001a8       __imp__strdup              00000001800051a8     ucrt:api-ms-win-crt-string-l1-1-0.dll
 0002:000001a8       __imp_strdup               00000001800051a8     ucrt:api-ms-win-crt-string-l1-1-0.dll
 0002:000001b0       __imp_strlen               00000001800051b0     ucrt:api-ms-win-crt-string-l1-1-0.dll
 0002:000001b8       __imp_strpbrk              00000001800051b8     ucrt:api-ms-win-crt-string-l1-1-0.dll
 0002:000001c0       __imp_strncpy              00000001800051c0     ucrt:api-ms-win-crt-string-l1-1-0.dll
 0002:000001c8       \177api-ms-win-crt-string-l1-1-0_NULL_THUNK_DATA 00000001800051c8     ucrt:api-ms-win-crt-string-l1-1-0.dll
 0002:000001d0       __guard_check_icall_fptr   00000001800051d0     MSVCRT:guard_support.obj
 0002:000001d8       __guard_xfg_check_icall_fptr 00000001800051d8     MSVCRT:guard_support.obj
 0002:000001e0       __guard_dispatch_icall_fptr 00000001800051e0     MSVCRT:guard_support.obj
 0002:000001e8       __guard_xfg_dispatch_icall_fptr 00000001800051e8     MSVCRT:guard_support.obj
 0002:000001f0       __guard_xfg_table_dispatch_icall_fptr 00000001800051f0     MSVCRT:guard_support.obj
 0002:000001f8       __castguard_check_failure_os_handled_fptr 00000001800051f8     MSVCRT:guard_support.obj
 0002:00000200       __guard_memcpy_fptr        0000000180005200     vcruntime:softmemtag.obj
 0002:00000208       __xc_a                     0000000180005208     MSVCRT:initializers.obj
 0002:00000210       __xc_z                     0000000180005210     MSVCRT:initializers.obj
 0002:00000218       __xi_a                     0000000180005218     MSVCRT:initializers.obj
 0002:00000228       __xi_z                     0000000180005228     MSVCRT:initializers.obj
 0002:00000230       __xl_a                     0000000180005230     MSVCRT:tlssup.obj
 0002:00000238       __xl_z                     0000000180005238     MSVCRT:tlssup.obj
 0002:00000240       __xp_a                     0000000180005240     MSVCRT:initializers.obj
 0002:00000248       __xp_z                     0000000180005248     MSVCRT:initializers.obj
 0002:00000250       __xt_a                     0000000180005250     MSVCRT:initializers.obj
 0002:00000258       __xt_z                     0000000180005258     MSVCRT:initializers.obj
 0002:00000260       g_refKindStr               0000000180005260     libsuspendthrd003.obj
 0002:00000410       ??_C@_09BPLDFGCI@unknown_0@ 0000000180005410     libsuspendthrd003.obj
 0002:00000420       ??_C@_0BL@FPNMECJD@JVMTI_HEAP_REFERENCE_CLASS@ 0000000180005420     libsuspendthrd003.obj
 0002:00000440       ??_C@_0BL@FKGKKLNM@JVMTI_HEAP_REFERENCE_FIELD@ 0000000180005440     libsuspendthrd003.obj
 0002:00000460       ??_C@_0CD@CAEHCFJF@JVMTI_HEAP_REFERENCE_ARRAY_ELEM@ 0000000180005460     libsuspendthrd003.obj
 0002:00000488       ??_C@_0CC@DNEBMCNK@JVMTI_HEAP_REFERENCE_CLASS_LOAD@ 0000000180005488     libsuspendthrd003.obj
 0002:000004b0       ??_C@_0BN@CJMIPEBB@JVMTI_HEAP_REFERENCE_SIGNERS@ 00000001800054b0     libsuspendthrd003.obj
 0002:000004d0       ??_C@_0CH@HBOIDPEB@JVMTI_HEAP_REFERENCE_PROTECTION@ 00000001800054d0     libsuspendthrd003.obj
 0002:000004f8       ??_C@_0BP@MDKGDGKL@JVMTI_HEAP_REFERENCE_INTERFACE@ 00000001800054f8     libsuspendthrd003.obj
 0002:00000518       ??_C@_0CC@JJMIHNJH@JVMTI_HEAP_REFERENCE_STATIC_FIE@ 0000000180005518     libsuspendthrd003.obj
 0002:00000540       ??_C@_0CD@IDHEEGID@JVMTI_HEAP_REFERENCE_CONSTANT_P@ 0000000180005540     libsuspendthrd003.obj
 0002:00000568       ??_C@_0CA@EFFCHNG@JVMTI_HEAP_REFERENCE_SUPERCLASS@ 0000000180005568     libsuspendthrd003.obj
 0002:00000588       ??_C@_0L@PCDFHGCJ@unknown_11@ 0000000180005588     libsuspendthrd003.obj
 0002:00000598       ??_C@_0L@NJBICFOK@unknown_12@ 0000000180005598     libsuspendthrd003.obj
 0002:000005a8       ??_C@_0L@MAADBEKL@unknown_13@ 00000001800055a8     libsuspendthrd003.obj
 0002:000005b8       ??_C@_0L@IPECICGM@unknown_14@ 00000001800055b8     libsuspendthrd003.obj
 0002:000005c8       ??_C@_0L@JGFJLDCN@unknown_15@ 00000001800055c8     libsuspendthrd003.obj
 0002:000005d8       ??_C@_0L@LNHEOAOO@unknown_16@ 00000001800055d8     libsuspendthrd003.obj
 0002:000005e8       ??_C@_0L@KEGPNBKP@unknown_17@ 00000001800055e8     libsuspendthrd003.obj
 0002:000005f8       ??_C@_0L@CDPHMNGA@unknown_18@ 00000001800055f8     libsuspendthrd003.obj
 0002:00000608       ??_C@_0L@DKOMPMCB@unknown_19@ 0000000180005608     libsuspendthrd003.obj
 0002:00000618       ??_C@_0L@OJGIPJDB@unknown_20@ 0000000180005618     libsuspendthrd003.obj
 0002:00000628       ??_C@_0CA@KAOFNDEM@JVMTI_HEAP_REFERENCE_JNI_GLOBAL@ 0000000180005628     libsuspendthrd003.obj
 0002:00000648       ??_C@_0CC@HPFAJBK@JVMTI_HEAP_REFERENCE_SYSTEM_CLA@ 0000000180005648     libsuspendthrd003.obj
 0002:00000670       ??_C@_0BN@FDEGFOHC@JVMTI_HEAP_REFERENCE_MONITOR@ 0000000180005670     libsuspendthrd003.obj
 0002:00000690       ??_C@_0CB@HKIBCMAJ@JVMTI_HEAP_REFERENCE_STACK_LOCA@ 0000000180005690     libsuspendthrd003.obj
 0002:000006b8       ??_C@_0BP@EAACMMOE@JVMTI_HEAP_REFERENCE_JNI_LOCAL@ 00000001800056b8     libsuspendthrd003.obj
 0002:000006d8       ??_C@_0BM@IJDEOGOE@JVMTI_HEAP_REFERENCE_THREAD@ 00000001800056d8     libsuspendthrd003.obj
 0002:000006f8       ??_C@_0BL@EDGPPKC@JVMTI_HEAP_REFERENCE_OTHER@ 00000001800056f8     libsuspendthrd003.obj
 0002:00000714       ??_C@_04BCJPDBDA@Code@     0000000180005714     libsuspendthrd003.obj
 0002:00000720       ??_C@_0BA@OCLMCFKC@LineNumberTable@ 0000000180005720     libsuspendthrd003.obj
 0002:00000730       ??_C@_0BD@CPAEPILC@LocalVariableTable@ 0000000180005730     libsuspendthrd003.obj
 0002:00000748       ??_C@_0BH@NMBDNHBD@LocalVariableTypeTable@ 0000000180005748     libsuspendthrd003.obj
 0002:00000760       ??_C@_0O@HIHEEDNJ@StackMapTable@ 0000000180005760     libsuspendthrd003.obj
 0002:00000770       ??_C@_0L@HCDIAMJG@?9?5?$CFs?0?5?$CFd?3?5@ 0000000180005770     libsuspendthrd003.obj
 0002:00000780       ??_C@_0JI@HLPECLFI@?$CD?5?4?4?4?6?$CD?5ERROR?3?5too?5many?5complai@ 0000000180005780     libsuspendthrd003.obj
 0002:00000820       ??_C@_0ED@JNEKCCOB@The?5following?5fake?5exception?5st@ 0000000180005820     libsuspendthrd003.obj
 0002:00000868       ??_C@_0CN@FCNMDFBH@nsk?4share?4Fake_Exception_for_RU@ 0000000180005868     libsuspendthrd003.obj
 0002:00000898       ??_C@_08PGFFNAEI@?$CI?$CFs?3?$CFd?$CJ?5@ 0000000180005898     libsuspendthrd003.obj
 0002:000008a8       ??_C@_0DP@IENMAEGI@s?2test?2hotspot?2jtreg?2vmTestbase@ 00000001800058a8     libsuspendthrd003.obj
 0002:000008e8       ??_C@_0BL@NDJLFFJB@?7at?5nsk_lvcomplain?$CI?$CFs?3?$CFd?$CJ?6@ 00000001800058e8     libsuspendthrd003.obj
 0002:00000908       ??_C@_0BC@JOOKAFKF@?$CD?5ERROR?3?5?$CFs?0?5?$CFd?3?5@ 0000000180005908     libsuspendthrd003.obj
 0002:00000920       ??_C@_09KJEAHMEH@?$CD?5ERROR?3?5@ 0000000180005920     libsuspendthrd003.obj
 0002:0000092c       ??_C@_02GPIOPFAK@?$DO?$DO@ 000000018000592c     libsuspendthrd003.obj
 0002:00000930       ??_C@_02FODMEDOG@?$DM?$DM@ 0000000180005930     libsuspendthrd003.obj
 0002:00000934       ??_C@_02DJGKEECL@?4?4@     0000000180005934     libsuspendthrd003.obj
 0002:00000938       ??_C@_0O@CJPGJOAF@?9?5?$CFs?0?5?$CFd?3?5?$CFs?5@ 0000000180005938     libsuspendthrd003.obj
 0002:00000948       ??_C@_0CB@IAKPDOIC@?$CD?5?5?5verified?5assertion?5is?5FALSE@ 0000000180005948     libsuspendthrd003.obj
 0002:00000970       ??_C@_0CO@LGONDEPD@stdout?3?5fflush?5failed?5?9?5err?$DN?$CFd?5@ 0000000180005970     libsuspendthrd003.obj
 0002:000009a0       ??_C@_0CO@KBGKJPBD@stderr?3?5fflush?5failed?5?9?5err?$DN?$CFd?5@ 00000001800059a0     libsuspendthrd003.obj
 0002:000009d0       ??_C@_06PAOMPDJH@?$DMnone?$DO@ 00000001800059d0     libsuspendthrd003.obj
 0002:000009d8       ??_C@_06PHAKILGJ@?5ALIVE@  00000001800059d8     libsuspendthrd003.obj
 0002:000009e0       ??_C@_0M@OFKKEJHG@?5TERMINATED@ 00000001800059e0     libsuspendthrd003.obj
 0002:000009f0       ??_C@_09JDCMELJI@?5RUNNABLE@ 00000001800059f0     libsuspendthrd003.obj
 0002:00000a00       ??_C@_08OAHMLBPA@?5WAITING@ 0000000180005a00     libsuspendthrd003.obj
 0002:00000a10       ??_C@_0BG@GOEBACGE@?5WAITING_INDEFINITELY@ 0000000180005a10     libsuspendthrd003.obj
 0002:00000a28       ??_C@_0BG@CCLPBKFG@?5WAITING_WITH_TIMEOUT@ 0000000180005a28     libsuspendthrd003.obj
 0002:00000a40       ??_C@_09DEFAFODN@?5SLEEPING@ 0000000180005a40     libsuspendthrd003.obj
 0002:00000a50       ??_C@_0BA@EIDDAKGK@?5IN_OBJECT_WAIT@ 0000000180005a50     libsuspendthrd003.obj
 0002:00000a60       ??_C@_07GIPIPEAD@?5PARKED@ 0000000180005a60     libsuspendthrd003.obj
 0002:00000a68       ??_C@_0BK@LNIHGEJF@?5BLOCKED_ON_MONITOR_ENTER@ 0000000180005a68     libsuspendthrd003.obj
 0002:00000a88       ??_C@_0L@MOBKJCJD@?5SUSPENDED@ 0000000180005a88     libsuspendthrd003.obj
 0002:00000a98       ??_C@_0N@CPMJCKAP@?5INTERRUPTED@ 0000000180005a98     libsuspendthrd003.obj
 0002:00000aa8       ??_C@_0L@PEJNJEEC@?5IN_NATIVE@ 0000000180005aa8     libsuspendthrd003.obj
 0002:00000ab8       ??_C@_0BB@JCNMKLLK@JVMTI_ERROR_NONE@ 0000000180005ab8     libsuspendthrd003.obj
 0002:00000ad0       ??_C@_0BL@LDIMKLPH@JVMTI_ERROR_INVALID_THREAD@ 0000000180005ad0     libsuspendthrd003.obj
 0002:00000af0       ??_C@_0CB@PJFPAIKJ@JVMTI_ERROR_INVALID_THREAD_GROU@ 0000000180005af0     libsuspendthrd003.obj
 0002:00000b18       ??_C@_0BN@LLMKHMNF@JVMTI_ERROR_INVALID_PRIORITY@ 0000000180005b18     libsuspendthrd003.obj
 0002:00000b38       ??_C@_0CB@MBOFKAGB@JVMTI_ERROR_THREAD_NOT_SUSPENDE@ 0000000180005b38     libsuspendthrd003.obj
 0002:00000b60       ??_C@_0BN@FABOLPBI@JVMTI_ERROR_THREAD_SUSPENDED@ 0000000180005b60     libsuspendthrd003.obj
 0002:00000b80       ??_C@_0BN@FDGNOBJM@JVMTI_ERROR_THREAD_NOT_ALIVE@ 0000000180005b80     libsuspendthrd003.obj
 0002:00000ba0       ??_C@_0BL@GOBIFKNJ@JVMTI_ERROR_INVALID_OBJECT@ 0000000180005ba0     libsuspendthrd003.obj
 0002:00000bc0       ??_C@_0BK@FCMAJPPC@JVMTI_ERROR_INVALID_CLASS@ 0000000180005bc0     libsuspendthrd003.obj
 0002:00000be0       ??_C@_0BP@IKLLBKEB@JVMTI_ERROR_CLASS_NOT_PREPARED@ 0000000180005be0     libsuspendthrd003.obj
 0002:00000c00       ??_C@_0BN@KLPPLKG@JVMTI_ERROR_INVALID_METHODID@ 0000000180005c00     libsuspendthrd003.obj
 0002:00000c20       ??_C@_0BN@BCEKOKND@JVMTI_ERROR_INVALID_LOCATION@ 0000000180005c20     libsuspendthrd003.obj
 0002:00000c40       ??_C@_0BM@DFDGPME@JVMTI_ERROR_INVALID_FIELDID@ 0000000180005c40     libsuspendthrd003.obj
 0002:00000c60       ??_C@_0BL@NELIEPEC@JVMTI_ERROR_NO_MORE_FRAMES@ 0000000180005c60     libsuspendthrd003.obj
 0002:00000c80       ??_C@_0BJ@BDBECFDM@JVMTI_ERROR_OPAQUE_FRAME@ 0000000180005c80     libsuspendthrd003.obj
 0002:00000ca0       ??_C@_0BK@MIIFNLOB@JVMTI_ERROR_TYPE_MISMATCH@ 0000000180005ca0     libsuspendthrd003.obj
 0002:00000cc0       ??_C@_0BJ@HPCAOILC@JVMTI_ERROR_INVALID_SLOT@ 0000000180005cc0     libsuspendthrd003.obj
 0002:00000ce0       ??_C@_0BG@CHILOPNI@JVMTI_ERROR_DUPLICATE@ 0000000180005ce0     libsuspendthrd003.obj
 0002:00000cf8       ??_C@_0BG@DIEMLHKM@JVMTI_ERROR_NOT_FOUND@ 0000000180005cf8     libsuspendthrd003.obj
 0002:00000d10       ??_C@_0BM@NHMCKHOB@JVMTI_ERROR_INVALID_MONITOR@ 0000000180005d10     libsuspendthrd003.obj
 0002:00000d30       ??_C@_0BO@PPEDAJGL@JVMTI_ERROR_NOT_MONITOR_OWNER@ 0000000180005d30     libsuspendthrd003.obj
 0002:00000d50       ??_C@_0BG@FCAIPEID@JVMTI_ERROR_INTERRUPT@ 0000000180005d50     libsuspendthrd003.obj
 0002:00000d68       ??_C@_0CB@EGDBNKOI@JVMTI_ERROR_INVALID_CLASS_FORMA@ 0000000180005d68     libsuspendthrd003.obj
 0002:00000d90       ??_C@_0CG@DGKOGIAL@JVMTI_ERROR_CIRCULAR_CLASS_DEFI@ 0000000180005d90     libsuspendthrd003.obj
 0002:00000db8       ??_C@_0BP@ICEALPKC@JVMTI_ERROR_FAILS_VERIFICATION@ 0000000180005db8     libsuspendthrd003.obj
 0002:00000dd8       ??_C@_0DC@JDACLMIO@JVMTI_ERROR_UNSUPPORTED_REDEFIN@ 0000000180005dd8     libsuspendthrd003.obj
 0002:00000e10       ??_C@_0DE@GKDKNOMJ@JVMTI_ERROR_UNSUPPORTED_REDEFIN@ 0000000180005e10     libsuspendthrd003.obj
 0002:00000e48       ??_C@_0BO@LAFKIOG@JVMTI_ERROR_INVALID_TYPESTATE@ 0000000180005e48     libsuspendthrd003.obj
 0002:00000e68       ??_C@_0DH@INDGCLLB@JVMTI_ERROR_UNSUPPORTED_REDEFIN@ 0000000180005e68     libsuspendthrd003.obj
 0002:00000ea0       ??_C@_0DE@NHEOMMGI@JVMTI_ERROR_UNSUPPORTED_REDEFIN@ 0000000180005ea0     libsuspendthrd003.obj
 0002:00000ed8       ??_C@_0CA@EKPNJOEP@JVMTI_ERROR_UNSUPPORTED_VERSION@ 0000000180005ed8     libsuspendthrd003.obj
 0002:00000ef8       ??_C@_0BN@OFFMAHHL@JVMTI_ERROR_NAMES_DONT_MATCH@ 0000000180005ef8     libsuspendthrd003.obj
 0002:00000f18       ??_C@_0DN@HHBBLAKE@JVMTI_ERROR_UNSUPPORTED_REDEFIN@ 0000000180005f18     libsuspendthrd003.obj
 0002:00000f58       ??_C@_0DO@HMBGBGNA@JVMTI_ERROR_UNSUPPORTED_REDEFIN@ 0000000180005f58     libsuspendthrd003.obj
 0002:00000f98       ??_C@_0BP@PBECGKHJ@JVMTI_ERROR_UNMODIFIABLE_CLASS@ 0000000180005f98     libsuspendthrd003.obj
 0002:00000fb8       ??_C@_0BK@CANILEHF@JVMTI_ERROR_NOT_AVAILABLE@ 0000000180005fb8     libsuspendthrd003.obj
 0002:00000fd8       ??_C@_0CE@INJKMEFK@JVMTI_ERROR_MUST_POSSESS_CAPABI@ 0000000180005fd8     libsuspendthrd003.obj
 0002:00001000       ??_C@_0BJ@LBFPFPDM@JVMTI_ERROR_NULL_POINTER@ 0000000180006000     libsuspendthrd003.obj
 0002:00001020       ??_C@_0BP@CHJPNNEM@JVMTI_ERROR_ABSENT_INFORMATION@ 0000000180006020     libsuspendthrd003.obj
 0002:00001040       ??_C@_0BP@OMFMNLC@JVMTI_ERROR_INVALID_EVENT_TYPE@ 0000000180006040     libsuspendthrd003.obj
 0002:00001060       ??_C@_0BN@BIBNPHHO@JVMTI_ERROR_ILLEGAL_ARGUMENT@ 0000000180006060     libsuspendthrd003.obj
 0002:00001080       ??_C@_0BK@KKNDHDCE@JVMTI_ERROR_NATIVE_METHOD@ 0000000180006080     libsuspendthrd003.obj
 0002:000010a0       ??_C@_0BK@PMKCFHAE@JVMTI_ERROR_OUT_OF_MEMORY@ 00000001800060a0     libsuspendthrd003.obj
 0002:000010c0       ??_C@_0BK@NNJBDMNB@JVMTI_ERROR_ACCESS_DENIED@ 00000001800060c0     libsuspendthrd003.obj
 0002:000010e0       ??_C@_0BI@GHECLMNC@JVMTI_ERROR_WRONG_PHASE@ 00000001800060e0     libsuspendthrd003.obj
 0002:000010f8       ??_C@_0BF@OLIHJOII@JVMTI_ERROR_INTERNAL@ 00000001800060f8     libsuspendthrd003.obj
 0002:00001110       ??_C@_0BO@EOHGKJHI@JVMTI_ERROR_UNATTACHED_THREAD@ 0000000180006110     libsuspendthrd003.obj
 0002:00001130       ??_C@_0CA@LKHFDACL@JVMTI_ERROR_INVALID_ENVIRONMENT@ 0000000180006130     libsuspendthrd003.obj
 0002:00001150       ??_C@_0BA@MMFHLOKK@?$DMunknown?5error?$DO@ 0000000180006150     libsuspendthrd003.obj
 0002:00001160       ??_C@_0CF@CBHOKDB@throwable?5?$DN?5jni?9?$DOExceptionOccur@ 0000000180006160     libsuspendthrd003.obj
 0002:00001188       ??_C@_03OFAPEBGM@?$CFs?6@  0000000180006188     libsuspendthrd003.obj
 0002:00001190       ??_C@_0DM@LPIGEGNJ@s?2test?2hotspot?2jtreg?2vmTestbase@ 0000000180006190     libsuspendthrd003.obj
 0002:000011d0       ??_C@_0CC@NFCNPEPK@Exception?5in?5JNI?5call?5?$CIcleared?$CJ@ 00000001800061d0     libsuspendthrd003.obj
 0002:000011f8       ??_C@_0BJ@IBAKFIKF@jni?9?$DOExceptionDescribe?$CI?$CJ@ 00000001800061f8     libsuspendthrd003.obj
 0002:00001218       ??_C@_0BG@GGKALKMH@jni?9?$DOExceptionClear?$CI?$CJ@ 0000000180006218     libsuspendthrd003.obj
 0002:00001230       ??_C@_0CF@JMGFGJLJ@?$CD?5?5?5verified?5JNI?5assertion?5is?5F@ 0000000180006230     libsuspendthrd003.obj
 0002:00001258       ??_C@_07KBAMPNJK@verbose@  0000000180006258     libsuspendthrd003.obj
 0002:00001260       ??_C@_0DN@PKJBOLAP@nsk_jvmti_parseOptions?$CI?$CJ?3?5unexp@ 0000000180006260     libsuspendthrd003.obj
 0002:000012a0       ??_C@_05IMBNNINJ@trace@    00000001800062a0     libsuspendthrd003.obj
 0002:000012a8       ??_C@_0DD@BJKGNDMB@nsk_jvmti_parseOptions?$CI?$CJ?3?5no?5va@ 00000001800062a8     libsuspendthrd003.obj
 0002:000012dc       ??_C@_04CGFJFPFD@none@     00000001800062dc     libsuspendthrd003.obj
 0002:000012e4       ??_C@_06BMELKFMA@before@   00000001800062e4     libsuspendthrd003.obj
 0002:000012ec       ??_C@_05CMKPCFDK@after@    00000001800062ec     libsuspendthrd003.obj
 0002:000012f4       ??_C@_03NFKEKGGK@all@      00000001800062f4     libsuspendthrd003.obj
 0002:000012f8       ??_C@_0DM@NDNJGJKE@nsk_jvmti_parseOptions?$CI?$CJ?3?5uexpe@ 00000001800062f8     libsuspendthrd003.obj
 0002:00001338       ??_C@_08NBBJKJO@waittime@  0000000180006338     libsuspendthrd003.obj
 0002:00001348       ??_C@_0DO@CMHGAOHC@nsk_jvmti_parseOptions?$CI?$CJ?3?5not?5i@ 0000000180006348     libsuspendthrd003.obj
 0002:00001388       ??_C@_0DL@LNMPBDLN@nsk_jvmti_parseOptions?$CI?$CJ?3?5negat@ 0000000180006388     libsuspendthrd003.obj
 0002:000013c8       ??_C@_0DA@GMFJNOJH@nsk_jvmti_parseOptions?$CI?$CJ?3?5unkno@ 00000001800063c8     libsuspendthrd003.obj
 0002:000013f8       ??_C@_0CO@CCIAMEAN@nsk_jvmti_parseOptions?$CI?$CJ?3?5found@ 00000001800063f8     libsuspendthrd003.obj
 0002:00001428       ??_C@_0CJ@OEGPCGDL@nsk_jvmti_parseOptions?$CI?$CJ?3?5out?5o@ 0000000180006428     libsuspendthrd003.obj
 0002:00001458       ??_C@_0DI@NMBHPGGF@nsk_jvmti_parseOptions?$CI?$CJ?3?5too?5m@ 0000000180006458     libsuspendthrd003.obj
 0002:00001490       ??_C@_03POGCGECB@?5?0?$HO@ 0000000180006490     libsuspendthrd003.obj
 0002:00001498       ??_C@_0CB@MLNJNCLJ@?5?5jvmti?5error?3?5code?$DN?$CFd?0?5name?$DN?$CFs@ 0000000180006498     libsuspendthrd003.obj
 0002:000014c0       ??_C@_0CD@OHBGDKMK@?$CD?5?5?5jvmti?5error?3?5code?$DN?$CFd?0?5name?$DN@ 00000001800064c0     libsuspendthrd003.obj
 0002:000014e8       ??_C@_0CG@JNNCGPHB@?$CD?5?5?5error?5expected?3?5code?$DN?$CFd?0?5na@ 00000001800064e8     libsuspendthrd003.obj
 0002:00001510       ??_C@_0EB@IMGKPCGE@?$CIstr_obj?5?$DN?5jni?9?$DONewStringUTF?$CIco@ 0000000180006510     libsuspendthrd003.obj
 0002:00001560       ??_C@_0EA@HFOGGBCC@s?2test?2hotspot?2jtreg?2vmTestbase@ 0000000180006560     libsuspendthrd003.obj
 0002:000015a0       ??_C@_05KKCIMGE@error@     00000001800065a0     libsuspendthrd003.obj
 0002:000015a8       ??_C@_0CJ@JACLEAA@Test?5failed?5by?5setFailStatus?$CI?$CJ?4@ 00000001800065a8     libsuspendthrd003.obj
 0002:000015d8       ??_C@_0BD@HGNAOMCP@agent_data_monitor@ 00000001800065d8     libsuspendthrd003.obj
 0002:000015f0       ??_C@_0EB@OGCLGKLN@javaVM?9?$DOGetEnv?$CI?$CIvoid?5?$CK?$CK?$CJ?$CGjvmti_@ 00000001800065f0     libsuspendthrd003.obj
 0002:00001640       ??_C@_0EA@PNBCDMOA@s?2test?2hotspot?2jtreg?2vmTestbase@ 0000000180006640     libsuspendthrd003.obj
 0002:00001680       ??_C@_0CI@DDPIFBGM@init_agent_data?$CIjvmti_env?0?5?$CGage@ 0000000180006680     libsuspendthrd003.obj
 0002:000016a8       ??_C@_0DI@ILAHDLMP@?$CI?$CKagentThreadProc?$CJ?$CIjvmti_env?0?5a@ 00000001800066a8     libsuspendthrd003.obj
 0002:000016e0       ??_C@_0BD@KDBALNLB@JVMTI?5agent?5thread@ 00000001800066e0     libsuspendthrd003.obj
 0002:000016f8       ??_C@_0BB@NOKBFPFO@java?1lang?1Thread@ 00000001800066f8     libsuspendthrd003.obj
 0002:0000170c       ??_C@_06FALKBLGB@?$DMinit?$DO@ 000000018000670c     libsuspendthrd003.obj
 0002:00001718       ??_C@_0BG@IKDDPPGD@?$CILjava?1lang?1String?$DL?$CJV@ 0000000180006718     libsuspendthrd003.obj
 0002:00001730       ??_C@_0EB@IFJBFEKC@?$CIthreadClass?5?$DN?5jni_env?9?$DOFindCla@ 0000000180006730     libsuspendthrd003.obj
 0002:00001780       ??_C@_0GF@FGFIBKKL@?$CIthreadCtor?5?$DN?5jni_env?9?$DOGetMetho@ 0000000180006780     libsuspendthrd003.obj
 0002:000017e8       ??_C@_0DN@NCPDJLOG@?$CIthreadName?5?$DN?5jni_env?9?$DONewStrin@ 00000001800067e8     libsuspendthrd003.obj
 0002:00001830       ??_C@_0FE@PFKODBGC@?$CIthreadObject?5?$DN?5jni_env?9?$DONewObj@ 0000000180006830     libsuspendthrd003.obj
 0002:00001890       ??_C@_0ED@HOBAHHJI@?$CIthreadGlobalRef?5?$DN?5jni_env?9?$DONew@ 0000000180006890     libsuspendthrd003.obj
 0002:000018e0       ??_C@_0FN@HNJJAHFC@jvmti_env?9?$DORunAgentThread?$CIagent@ 00000001800068e0     libsuspendthrd003.obj
 0002:00001940       ??_C@_0EA@MOJDNKDF@Debuggee?5status?5sync?5aborted?5be@ 0000000180006940     libsuspendthrd003.obj
 0002:00001980       ??_C@_0CO@PGPGMHBJ@No?5status?5sync?5occured?5for?5time@ 0000000180006980     libsuspendthrd003.obj
 0002:000019b0       ??_C@_0CL@DOEBDPKJ@Debuggee?5was?5not?5suspended?5on?5s@ 00000001800069b0     libsuspendthrd003.obj
 0002:000019e0       ??_C@_0EA@EEOEJAEN@status?5?$DN?5syncDebuggeeStatus?$CIjni@ 00000001800069e0     libsuspendthrd003.obj
 0002:00001a20       ??_C@_0BL@JBCFNBMB@nsk_jvmti_resetAgentData?$CI?$CJ@ 0000000180006a20     libsuspendthrd003.obj
 0002:00001a40       ??_C@_0BA@OEGNKEHK@name?5?$CB?$DN?5nullptr@ 0000000180006a40     libsuspendthrd003.obj
 0002:00001a50       ??_C@_0CL@BAHDCEOM@jvmti_env?9?$DOGetAllThreads?$CI?$CGcount@ 0000000180006a50     libsuspendthrd003.obj
 0002:00001a80       ??_C@_0CM@KHOAGNIJ@jvmti_env?9?$DOGetThreadInfo?$CIthread@ 0000000180006a80     libsuspendthrd003.obj
 0002:00001ab0       ??_C@_0DB@JOGMPONN@jvmti_env?9?$DODeallocate?$CI?$CIunsigned@ 0000000180006ab0     libsuspendthrd003.obj
 0002:00001ae8       ??_C@_0CP@KMNIFKEK@jvmti_env?9?$DODeallocate?$CI?$CIunsigned@ 0000000180006ae8     libsuspendthrd003.obj
 0002:00001b20       ??_C@_0EI@EJCFGEKG@?$CIfoundThread?5?$DN?5?$CIjthread?$CJ?5jni_en@ 0000000180006b20     libsuspendthrd003.obj
 0002:00001b70       ??_C@_0EL@LPBEELIP@s?2test?2hotspot?2jtreg?2vmTestbase@ 0000000180006b70     libsuspendthrd003.obj
 0002:00001bc0       ??_C@_0CK@JDAMFDMJ@jvmti?9?$DOSetTag?$CIo?0?5tag?$CJ?5?$DN?$DN?5JVMTI_@ 0000000180006bc0     libsuspendthrd003.obj
 0002:00001bf0       ??_C@_0CC@DAMNHKNI@Can?8t?5set?5tag?5?$CFli?5for?5object?5?$CFl@ 0000000180006bf0     libsuspendthrd003.obj
 0002:00001c18       ??_C@_0DL@HAJPNKEF@jvmti?9?$DOGetObjectHashCode?$CIo?0?5?$CGha@ 0000000180006c18     libsuspendthrd003.obj
 0002:00001c58       ??_C@_0BL@JFPIEOBF@Can?8t?5get?5hash?5object?5?$CFlx?6@ 0000000180006c58     libsuspendthrd003.obj
 0002:00001c78       ??_C@_0BG@DICPHBKN@setTag?3?5?$CF08x?5?$DM?9?5?$CF?53li@ 0000000180006c78     libsuspendthrd003.obj
 0002:00001c90       ??_C@_0DH@FCEEBDMJ@?$CIs?5?$DN?5jni?9?$DOGetStringUTFChars?$CIsIn@ 0000000180006c90     libsuspendthrd003.obj
 0002:00001cc8       ??_C@_0BJ@OKKGHDCN@Can?8t?5get?5string?5at?5?$CF?$CDp?6@ 0000000180006cc8     libsuspendthrd003.obj
 0002:00001ce8       ??_C@_0BP@EKFLGGFJ@Can?8t?5get?5string?5at?5?$CF?$CDp?3?5null?6@ 0000000180006ce8     libsuspendthrd003.obj
 0002:00001d08       ??_C@_06ICODBHCL@?5?1?1?5?$CFs@ 0000000180006d08     libsuspendthrd003.obj
 0002:00001d10       ??_C@_0DB@KGFPLEGO@?$CIr?5?$DN?5jvmti?9?$DOGetTag?$CIo?0?5?$CGtag?$CJ?$CJ?5?$DN?$DN@ 0000000180006d10     libsuspendthrd003.obj
 0002:00001d48       ??_C@_0CO@PDAGBCGJ@Can?8t?5GetTag?5for?5object?5?$CFlx?4?5Re@ 0000000180006d48     libsuspendthrd003.obj
 0002:00001d78       ??_C@_0CH@HPEODOHC@TEST_BUG?3?5Max?4?5number?5of?5refs?5r@ 0000000180006d78     libsuspendthrd003.obj
 0002:00001da0       ??_C@_0DI@PHFCABIM@?$CIr?5?$DN?5jvmti?9?$DOGetTag?$CIfrom?0?5?$CGtagFr@ 0000000180006da0     libsuspendthrd003.obj
 0002:00001dd8       ??_C@_0DI@MDEGFNKD@TEST_BUG?3?5Can?8t?5GetTag?5for?5obje@ 0000000180006dd8     libsuspendthrd003.obj
 0002:00001e10       ??_C@_0DE@MLELJAHM@?$CIr?5?$DN?5jvmti?9?$DOGetTag?$CIto?0?5?$CGtagTo?$CJ?$CJ@ 0000000180006e10     libsuspendthrd003.obj
 0002:00001e48       ??_C@_0BK@FLHGHEGH@Wait?5for?5thread?5to?5start?6@ 0000000180006e48     libsuspendthrd003.obj
 0002:00001e70       ??_C@_0FK@KEJALFHA@s?2test?2hotspot?2jtreg?2vmTestbase@ 0000000180006e70     libsuspendthrd003.obj
 0002:00001ed0       ??_C@_0N@KHCNHPIB@TestedThread@ 0000000180006ed0     libsuspendthrd003.obj
 0002:00001ee0       ??_C@_0BB@LECFLHJN@Find?5thread?3?5?$CFs?6@ 0000000180006ee0     libsuspendthrd003.obj
 0002:00001f00       ??_C@_0EA@GJLOKOPF@?$CItestedThread?5?$DN?5nsk_jvmti_threa@ 0000000180006f00     libsuspendthrd003.obj
 0002:00001f40       ??_C@_0BI@OFHDEFEM@?5?5?4?4?4?5found?5thread?3?5?$CFp?6@ 0000000180006f40     libsuspendthrd003.obj
 0002:00001f58       ??_C@_0BE@FGIAIPOM@Suspend?5thread?3?5?$CFp?6@ 0000000180006f58     libsuspendthrd003.obj
 0002:00001f70       ??_C@_0CD@PNHHKPAM@jvmti?9?$DOSuspendThread?$CItestedThre@ 0000000180006f70     libsuspendthrd003.obj
 0002:00001f98       ??_C@_0BO@MHPDHLNH@Let?5thread?5to?5run?5and?5finish?6@ 0000000180006f98     libsuspendthrd003.obj
 0002:00001fb8       ??_C@_0CB@JADEBEHF@Get?5state?5vector?5for?5thread?3?5?$CFp@ 0000000180006fb8     libsuspendthrd003.obj
 0002:00001fe0       ??_C@_0CM@OMAJINEK@jvmti?9?$DOGetThreadState?$CItestedThr@ 0000000180006fe0     libsuspendthrd003.obj
 0002:00002010       ??_C@_0CB@BKACHNJD@?5?5?4?4?4?5got?5state?5vector?3?5?$CFs?5?$CI?$CFd?$CJ@ 0000000180007010     libsuspendthrd003.obj
 0002:00002040       ??_C@_0EF@OONAFOJE@SuspendThread?$CI?$CJ?5does?5not?5turn?5o@ 0000000180007040     libsuspendthrd003.obj
 0002:00002088       ??_C@_0BD@IMGAGICA@Resume?5thread?3?5?$CFp?6@ 0000000180007088     libsuspendthrd003.obj
 0002:000020a0       ??_C@_0CC@OKFCGMH@jvmti?9?$DOResumeThread?$CItestedThrea@ 00000001800070a0     libsuspendthrd003.obj
 0002:000020c8       ??_C@_0BP@KJGLLBPM@INFO?3?5Late?5suspend?5thread?3?5?$CFp?6@ 00000001800070c8     libsuspendthrd003.obj
 0002:000020e8       ??_C@_0CD@KKLMNEFE@INFO?3?5Late?5suspend?5thread?5err?3?5@ 00000001800070e8     libsuspendthrd003.obj
 0002:00002110       ??_C@_0BO@GIDEAIPJ@INFO?3?5Late?5resume?5thread?3?5?$CFp?6@ 0000000180007110     libsuspendthrd003.obj
 0002:00002130       ??_C@_0BL@CLNCJLPF@Wait?5for?5thread?5to?5finish?6@ 0000000180007130     libsuspendthrd003.obj
 0002:00002150       ??_C@_0BJ@HHJICIEL@Delete?5thread?5reference?6@ 0000000180007150     libsuspendthrd003.obj
 0002:00002170       ??_C@_0CD@JEIIOPBJ@jni?9?$DODeleteGlobalRef?$CItestedThre@ 0000000180007170     libsuspendthrd003.obj
 0002:00002198       ??_C@_0BH@HPEOJMHL@Let?5debugee?5to?5finish?6@ 0000000180007198     libsuspendthrd003.obj
 0002:000021b0       ??_C@_0CA@MNKGCBCG@nsk_jvmti_parseOptions?$CIoptions?$CJ@ 00000001800071b0     libsuspendthrd003.obj
 0002:000021d0       ??_C@_0DN@MIAMNFPH@?$CIjvmti?5?$DN?5nsk_jvmti_createJVMTIE@ 00000001800071d0     libsuspendthrd003.obj
 0002:00002210       ??_C@_0CF@DFAKMCIB@jvmti?9?$DOAddCapabilities?$CI?$CGsuspend@ 0000000180007210     libsuspendthrd003.obj
 0002:00002238       ??_C@_0CL@PIACJIPK@nsk_jvmti_setAgentProc?$CIagentPro@ 0000000180007238     libsuspendthrd003.obj
 0002:00002280       ??_C@_1EC@JIJBPKFM@?$AAa?$AAp?$AAi?$AA?9?$AAm?$AAs?$AA?9?$AAw?$AAi?$AAn?$AA?9?$AAc?$AAo?$AAr?$AAe@ 0000000180007280     MSVCRT:thread_safe_statics.obj
 0002:000022c8       ??_C@_1BK@MGMFAEKH@?$AAk?$AAe?$AAr?$AAn?$AAe?$AAl?$AA3?$AA2?$AA?4?$AAd?$AAl?$AAl@ 00000001800072c8     MSVCRT:thread_safe_statics.obj
 0002:000022e8       ??_C@_0BJ@JEBJOJFJ@SleepConditionVariableCS@ 00000001800072e8     MSVCRT:thread_safe_statics.obj
 0002:00002308       ??_C@_0BJ@PGPPEPCC@WakeAllConditionVariable@ 0000000180007308     MSVCRT:thread_safe_statics.obj
 0002:00002328       _pDefaultRawDllMain        0000000180007328     MSVCRT:dll_dllmain.obj
 0002:00002328       _pRawDllMain               0000000180007328     MSVCRT:dll_dllmain.obj
 0002:00002330       __xmm@ffffffffffffffffffffffffffffffff 0000000180007330     MSVCRT:utility.obj
 0002:00002340       _load_config_used          0000000180007340     MSVCRT:loadcfg.obj
 0002:00002500       _tls_used                  0000000180007500     MSVCRT:tlssup.obj
 0002:00002528       __volatile_metadata        0000000180007528     <linker-defined>
 0002:00002900       __rtc_iaa                  0000000180007900     MSVCRT:initsect.obj
 0002:00002908       __rtc_izz                  0000000180007908     MSVCRT:initsect.obj
 0002:00002910       __rtc_taa                  0000000180007910     MSVCRT:initsect.obj
 0002:00002918       __rtc_tzz                  0000000180007918     MSVCRT:initsect.obj
 0002:00002920       _tls_start                 0000000180007920     MSVCRT:tlssup.obj
 0002:00002924       _Init_thread_epoch         0000000180007924     MSVCRT:thread_safe_statics.obj
 0002:00002928       _tls_end                   0000000180007928     MSVCRT:tlssup.obj
 0002:00002fd8       __IMPORT_DESCRIPTOR_KERNEL32 0000000180007fd8     kernel32:KERNEL32.dll
 0002:00002fec       __IMPORT_DESCRIPTOR_VCRUNTIME140 0000000180007fec     vcruntime:VCRUNTIME140.dll
 0002:00003000       __IMPORT_DESCRIPTOR_api-ms-win-crt-heap-l1-1-0 0000000180008000     ucrt:api-ms-win-crt-heap-l1-1-0.dll
 0002:00003014       __IMPORT_DESCRIPTOR_api-ms-win-crt-runtime-l1-1-0 0000000180008014     ucrt:api-ms-win-crt-runtime-l1-1-0.dll
 0002:00003028       __IMPORT_DESCRIPTOR_api-ms-win-crt-convert-l1-1-0 0000000180008028     ucrt:api-ms-win-crt-convert-l1-1-0.dll
 0002:0000303c       __IMPORT_DESCRIPTOR_api-ms-win-crt-stdio-l1-1-0 000000018000803c     ucrt:api-ms-win-crt-stdio-l1-1-0.dll
 0002:00003050       __IMPORT_DESCRIPTOR_api-ms-win-crt-string-l1-1-0 0000000180008050     ucrt:api-ms-win-crt-string-l1-1-0.dll
 0002:00003064       __NULL_IMPORT_DESCRIPTOR   0000000180008064     kernel32:KERNEL32.dll
 0003:00000030       _Init_global_epoch         0000000180009030     MSVCRT:thread_safe_statics.obj
 0003:00000040       __security_cookie          0000000180009040     MSVCRT:gs_cookie.obj
 0003:00000048       __security_cookie_complement 0000000180009048     MSVCRT:gs_cookie.obj
 0003:00000050       __scrt_native_dllmain_reason 0000000180009050     MSVCRT:utility.obj
 0003:00000058       __isa_available            0000000180009058     MSVCRT:cpu_disp.obj
 0003:0000005c       __isa_enabled              000000018000905c     MSVCRT:cpu_disp.obj
 0003:00000060       __memset_fast_string_threshold 0000000180009060     MSVCRT:cpu_disp.obj
 0003:00000068       __memset_nt_threshold      0000000180009068     MSVCRT:cpu_disp.obj
 0003:00000070       __scrt_ucrt_dll_is_in_use  0000000180009070     MSVCRT:ucrt_stubs.obj
 0003:00000080       g_wrongHeapCallbacks       0000000180009080     libsuspendthrd003.obj
 0003:00000100       g_szTagInfo                0000000180009100     libsuspendthrd003.obj
 0003:00002040       g_tagFlags                 000000018000b040     libsuspendthrd003.obj
 0003:00002428       g_refsToVerifyCnt          000000018000b428     libsuspendthrd003.obj
 0003:0000242c       g_fakeUserData             000000018000b42c     libsuspendthrd003.obj
 0003:00002430       g_tagVisitCount            000000018000b430     libsuspendthrd003.obj
 0003:000033d0       g_refsToVerify             000000018000c3d0     libsuspendthrd003.obj
 0003:0001aad0       g_userDataError            0000000180023ad0     libsuspendthrd003.obj
 0003:0001ac70       ?_OptionsStorage@?1??__local_stdio_printf_options@@9@4_KA 0000000180023c70     libsuspendthrd003.obj
 0003:0001b368       _tls_index                 0000000180024368     MSVCRT:tlssup.obj
 0003:0001b370       __scrt_current_native_startup_state 0000000180024370     MSVCRT:utility.obj
 0003:0001b378       __scrt_native_startup_lock 0000000180024378     MSVCRT:utility.obj
 0003:0001b3b8       __scrt_debugger_hook_flag  00000001800243b8     MSVCRT:utility_desktop.obj
 0003:0001b3c0       ?__type_info_root_node@@3U__type_info_node@@A 00000001800243c0     MSVCRT:tncleanup.obj
 0003:0001b3d0       ?_OptionsStorage@?1??__local_stdio_scanf_options@@9@4_KA 00000001800243d0     MSVCRT:default_local_stdio_options.obj
 0003:0001b3d8       __favor                    00000001800243d8     MSVCRT:cpu_disp.obj
 0003:0001b3e0       __dyn_tls_init_callback    00000001800243e0     <common>

 entry point at        0001:00003340

 Static symbols

 0000:fffd9000       .debug$S                   0000000180000000     suspendthrd003.exp
 0000:fffd9000       .debug$S                   0000000180000000     vcruntime:VCRUNTIME140.dll
 0000:fffd9000       .debug$S                   0000000180000000     vcruntime:VCRUNTIME140.dll
 0000:fffd9000       .debug$S                   0000000180000000     vcruntime:VCRUNTIME140.dll
 0000:fffd9000       .debug$S                   0000000180000000     vcruntime:VCRUNTIME140.dll
 0000:fffd9000       .debug$S                   0000000180000000     vcruntime:VCRUNTIME140.dll
 0000:fffd9000       .debug$S                   0000000180000000     vcruntime:VCRUNTIME140.dll
 0000:fffd9000       .debug$S                   0000000180000000     vcruntime:VCRUNTIME140.dll
 0000:fffd9000       .debug$S                   0000000180000000     ucrt:api-ms-win-crt-convert-l1-1-0.dll
 0000:fffd9000       .debug$S                   0000000180000000     ucrt:api-ms-win-crt-heap-l1-1-0.dll
 0000:fffd9000       .debug$S                   0000000180000000     ucrt:api-ms-win-crt-heap-l1-1-0.dll
 0000:fffd9000       .debug$S                   0000000180000000     ucrt:api-ms-win-crt-heap-l1-1-0.dll
 0000:fffd9000       .debug$S                   0000000180000000     ucrt:api-ms-win-crt-heap-l1-1-0.dll
 0000:fffd9000       .debug$S                   0000000180000000     ucrt:api-ms-win-crt-runtime-l1-1-0.dll
 0000:fffd9000       .debug$S                   0000000180000000     ucrt:api-ms-win-crt-runtime-l1-1-0.dll
 0000:fffd9000       .debug$S                   0000000180000000     ucrt:api-ms-win-crt-runtime-l1-1-0.dll
 0000:fffd9000       .debug$S                   0000000180000000     ucrt:api-ms-win-crt-runtime-l1-1-0.dll
 0000:fffd9000       .debug$S                   0000000180000000     ucrt:api-ms-win-crt-runtime-l1-1-0.dll
 0000:fffd9000       .debug$S                   0000000180000000     ucrt:api-ms-win-crt-runtime-l1-1-0.dll
 0000:fffd9000       .debug$S                   0000000180000000     ucrt:api-ms-win-crt-runtime-l1-1-0.dll
 0000:fffd9000       .debug$S                   0000000180000000     ucrt:api-ms-win-crt-runtime-l1-1-0.dll
 0000:fffd9000       .debug$S                   0000000180000000     ucrt:api-ms-win-crt-runtime-l1-1-0.dll
 0000:fffd9000       .debug$S                   0000000180000000     ucrt:api-ms-win-crt-runtime-l1-1-0.dll
 0000:fffd9000       .debug$S                   0000000180000000     ucrt:api-ms-win-crt-runtime-l1-1-0.dll
 0000:fffd9000       .debug$S                   0000000180000000     ucrt:api-ms-win-crt-runtime-l1-1-0.dll
 0000:fffd9000       .debug$S                   0000000180000000     ucrt:api-ms-win-crt-runtime-l1-1-0.dll
 0000:fffd9000       .debug$S                   0000000180000000     ucrt:api-ms-win-crt-runtime-l1-1-0.dll
 0000:fffd9000       .debug$S                   0000000180000000     ucrt:api-ms-win-crt-runtime-l1-1-0.dll
 0000:fffd9000       .debug$S                   0000000180000000     ucrt:api-ms-win-crt-runtime-l1-1-0.dll
 0000:fffd9000       .debug$S                   0000000180000000     ucrt:api-ms-win-crt-stdio-l1-1-0.dll
 0000:fffd9000       .debug$S                   0000000180000000     ucrt:api-ms-win-crt-stdio-l1-1-0.dll
 0000:fffd9000       .debug$S                   0000000180000000     ucrt:api-ms-win-crt-stdio-l1-1-0.dll
 0000:fffd9000       .debug$S                   0000000180000000     ucrt:api-ms-win-crt-stdio-l1-1-0.dll
 0000:fffd9000       .debug$S                   0000000180000000     ucrt:api-ms-win-crt-stdio-l1-1-0.dll
 0000:fffd9000       .debug$S                   0000000180000000     ucrt:api-ms-win-crt-stdio-l1-1-0.dll
 0000:fffd9000       .debug$S                   0000000180000000     ucrt:api-ms-win-crt-stdio-l1-1-0.dll
 0000:fffd9000       .debug$S                   0000000180000000     ucrt:api-ms-win-crt-stdio-l1-1-0.dll
 0000:fffd9000       .debug$S                   0000000180000000     ucrt:api-ms-win-crt-stdio-l1-1-0.dll
 0000:fffd9000       .debug$S                   0000000180000000     ucrt:api-ms-win-crt-stdio-l1-1-0.dll
 0000:fffd9000       .debug$S                   0000000180000000     ucrt:api-ms-win-crt-string-l1-1-0.dll
 0000:fffd9000       .debug$S                   0000000180000000     ucrt:api-ms-win-crt-string-l1-1-0.dll
 0000:fffd9000       .debug$S                   0000000180000000     ucrt:api-ms-win-crt-string-l1-1-0.dll
 0000:fffd9000       .debug$S                   0000000180000000     ucrt:api-ms-win-crt-string-l1-1-0.dll
 0000:fffd9000       .debug$S                   0000000180000000     ucrt:api-ms-win-crt-string-l1-1-0.dll
 0000:fffd9000       .debug$S                   0000000180000000     ucrt:api-ms-win-crt-string-l1-1-0.dll
 0000:fffd9000       .debug$S                   0000000180000000     ucrt:api-ms-win-crt-string-l1-1-0.dll
 0000:fffd9000       .debug$S                   0000000180000000     ucrt:api-ms-win-crt-string-l1-1-0.dll
 0000:fffd9000       .debug$S                   0000000180000000     kernel32:KERNEL32.dll
 0000:fffd9000       .debug$S                   0000000180000000     kernel32:KERNEL32.dll
 0000:fffd9000       .debug$S                   0000000180000000     kernel32:KERNEL32.dll
 0000:fffd9000       .debug$S                   0000000180000000     kernel32:KERNEL32.dll
 0000:fffd9000       .debug$S                   0000000180000000     kernel32:KERNEL32.dll
 0000:fffd9000       .debug$S                   0000000180000000     kernel32:KERNEL32.dll
 0000:fffd9000       .debug$S                   0000000180000000     kernel32:KERNEL32.dll
 0000:fffd9000       .debug$S                   0000000180000000     kernel32:KERNEL32.dll
 0000:fffd9000       .debug$S                   0000000180000000     kernel32:KERNEL32.dll
 0000:fffd9000       .debug$S                   0000000180000000     kernel32:KERNEL32.dll
 0000:fffd9000       .debug$S                   0000000180000000     kernel32:KERNEL32.dll
 0000:fffd9000       .debug$S                   0000000180000000     kernel32:KERNEL32.dll
 0000:fffd9000       .debug$S                   0000000180000000     kernel32:KERNEL32.dll
 0000:fffd9000       .debug$S                   0000000180000000     kernel32:KERNEL32.dll
 0000:fffd9000       .debug$S                   0000000180000000     kernel32:KERNEL32.dll
 0000:fffd9000       .debug$S                   0000000180000000     kernel32:KERNEL32.dll
 0000:fffd9000       .debug$S                   0000000180000000     kernel32:KERNEL32.dll
 0000:fffd9000       .debug$S                   0000000180000000     kernel32:KERNEL32.dll
 0000:fffd9000       .debug$S                   0000000180000000     kernel32:KERNEL32.dll
 0000:fffd9000       .debug$S                   0000000180000000     kernel32:KERNEL32.dll
 0000:fffd9000       .debug$S                   0000000180000000     kernel32:KERNEL32.dll
 0000:fffd9000       .debug$S                   0000000180000000     kernel32:KERNEL32.dll
 0000:fffd9000       .debug$S                   0000000180000000     kernel32:KERNEL32.dll
 0000:fffd9000       .debug$S                   0000000180000000     kernel32:KERNEL32.dll
 0000:fffd9000       .debug$S                   0000000180000000     kernel32:KERNEL32.dll
 0000:fffd9000       .debug$S                   0000000180000000     kernel32:KERNEL32.dll
 0000:fffd9000       .debug$S                   0000000180000000     kernel32:KERNEL32.dll
 0000:fffd9000       .debug$S                   0000000180000000     kernel32:KERNEL32.dll
 0001:00000f90       addRefToVerify             0000000180001f90 f   libsuspendthrd003.obj
 0001:00000ffc       agentProc                  0000000180001ffc f   libsuspendthrd003.obj
 0001:0000158c       agentThreadWrapper         000000018000258c f   libsuspendthrd003.obj
 0001:000016f8       check_option               00000001800026f8 f   libsuspendthrd003.obj
 0001:00001940       file_basename              0000000180002940 f   libsuspendthrd003.obj
 0001:00002824       startAgentThreadWrapper    0000000180003824 f   libsuspendthrd003.obj
 0001:00002b64       syncDebuggeeStatus         0000000180003b64 f   libsuspendthrd003.obj
 0001:00002e04       capture_previous_context   0000000180003e04 f   MSVCRT:gs_report.obj
 0001:00002e78       ?__scrt_initialize_thread_safe_statics@@YAHXZ 0000000180003e78 f   MSVCRT:thread_safe_statics.obj
 0001:00002f48       ?__scrt_uninitialize_thread_safe_statics@@YAXXZ 0000000180003f48 f   MSVCRT:thread_safe_statics.obj
 0001:00002ff0       $$000000                   0000000180003ff0     MSVCRT:amdsecgs.obj
 0001:00003020       ?dllmain_crt_dispatch@@YAHQEAUHINSTANCE__@@KQEAX@Z 0000000180004020 f   MSVCRT:dll_dllmain.obj
 0001:00003070       ?dllmain_crt_process_attach@@YAHQEAUHINSTANCE__@@QEAX@Z 0000000180004070 f   MSVCRT:dll_dllmain.obj
 0001:00003188       ?dllmain_crt_process_detach@@YAH_N@Z 0000000180004188 f   MSVCRT:dll_dllmain.obj
 0001:0000320c       ?dllmain_dispatch@@YAHQEAUHINSTANCE__@@KQEAX@Z 000000018000420c f   MSVCRT:dll_dllmain.obj
 0001:00003c30       $$000000                   0000000180004c30     MSVCRT:guard_dispatch.obj
 0001:00003c50       $$000000                   0000000180004c50     MSVCRT:guard_xfg_dispatch.obj
 0001:00003c66       ?fin$0@?0??dllmain_crt_process_attach@@YAHQEAUHINSTANCE__@@QEAX@Z@4HA 0000000180004c66 f   MSVCRT:dll_dllmain.obj
 0001:00003c7d       ?fin$0@?0??dllmain_crt_process_detach@@YAH_N@Z@4HA 0000000180004c7d f   MSVCRT:dll_dllmain.obj
 0001:00003c96       ?fin$1@?0??dllmain_crt_process_detach@@YAH_N@Z@4HA 0000000180004c96 f   MSVCRT:dll_dllmain.obj
 0001:00003caa       ?filt$0@?0??dllmain_dispatch@@YAHQEAUHINSTANCE__@@KQEAX@Z@4HA 0000000180004caa f   MSVCRT:dll_dllmain.obj
 0001:00003ce0       __scrt_is_nonwritable_in_current_image$filt$0 0000000180004ce0 f   MSVCRT:utility.obj
 0002:00000220       ?__scrt_initialize_tss_var@@3P6AHXZEA 0000000180005220     MSVCRT:thread_safe_statics.obj
 0002:00000340       ?opcLengths@@3QBEB         0000000180005340     libsuspendthrd003.obj
 0002:00002268       GS_ExceptionPointers       0000000180007268     MSVCRT:gs_report.obj
 0002:00002930       $unwind$fprintf            0000000180007930     libsuspendthrd003.obj
 0002:0000293c       $unwind$printf             000000018000793c     libsuspendthrd003.obj
 0002:00002948       $unwind$?NewObject@JNIEnv_@@QEAAPEAV_jobject@@PEAV_jclass@@PEAU_jmethodID@@ZZ 0000000180007948     libsuspendthrd003.obj
 0002:00002948       $unwind$nsk_lcomplain      0000000180007948     libsuspendthrd003.obj
 0002:00002948       $unwind$nsk_ldisplay       0000000180007948     libsuspendthrd003.obj
 0002:00002950       $unwind$?TranslateState@@YAPEBDH@Z 0000000180007950     libsuspendthrd003.obj
 0002:00002950       $unwind$nsk_jvmti_waitForSync 0000000180007950     libsuspendthrd003.obj
 0002:00002950       $unwind$nsk_lvdisplay      0000000180007950     libsuspendthrd003.obj
 0002:00002950       $unwind$_RTC_Initialize    0000000180007950     MSVCRT:initsect.obj
 0002:00002950       $unwind$_RTC_Terminate     0000000180007950     MSVCRT:initsect.obj
 0002:00002950       $unwind$?__scrt_initialize_thread_safe_statics@@YAHXZ 0000000180007950     MSVCRT:thread_safe_statics.obj
 0002:0000295c       $unwind$nsk_complain       000000018000795c     libsuspendthrd003.obj
 0002:0000295c       $unwind$nsk_printf         000000018000795c     libsuspendthrd003.obj
 0002:00002964       $unwind$nsk_lvcomplain     0000000180007964     libsuspendthrd003.obj
 0002:0000297c       $unwind$nsk_ltrace         000000018000797c     libsuspendthrd003.obj
 0002:0000297c       $unwind$__report_gsfailure 000000018000797c     MSVCRT:gs_report.obj
 0002:00002984       $unwind$nsk_lvtrace        0000000180007984     libsuspendthrd003.obj
 0002:00002984       $unwind$__raise_securityfailure 0000000180007984     MSVCRT:gs_report.obj
 0002:00002984       $unwind$__scrt_initialize_crt 0000000180007984     MSVCRT:utility.obj
 0002:00002984       $unwind$__scrt_initialize_onexit_tables 0000000180007984     MSVCRT:utility.obj
 0002:00002984       $unwind$__scrt_release_startup_lock 0000000180007984     MSVCRT:utility.obj
 0002:00002984       $unwind$__scrt_uninitialize_crt 0000000180007984     MSVCRT:utility.obj
 0002:00002984       $unwind$_onexit            0000000180007984     MSVCRT:utility.obj
 0002:0000298c       $unwind$nsk_lverify        000000018000798c     libsuspendthrd003.obj
 0002:0000299c       $unwind$nsk_vprintf        000000018000799c     libsuspendthrd003.obj
 0002:000029ac       $unwind$?nsk_jni_lverify@@YAHHPEAUJNIEnv_@@HQEBDH1ZZ 00000001800079ac     libsuspendthrd003.obj
 0002:000029c0       $unwind$?nsk_jni_check_exception@@YAHPEAUJNIEnv_@@QEBDH@Z 00000001800079c0     libsuspendthrd003.obj
 0002:000029dc       $unwind$nsk_jvmti_parseOptions 00000001800079dc     libsuspendthrd003.obj
 0002:000029f8       $unwind$nsk_jvmti_createJVMTIEnv 00000001800079f8     libsuspendthrd003.obj
 0002:00002a0c       $unwind$Java_nsk_jvmti_unit_FollowReferences_FollowRefObjects_resetTags 0000000180007a0c     libsuspendthrd003.obj
 0002:00002a0c       $unwind$addRefToVerify     0000000180007a0c     libsuspendthrd003.obj
 0002:00002a0c       $unwind$nsk_jvmti_resetAgentData 0000000180007a0c     libsuspendthrd003.obj
 0002:00002a0c       $unwind$nsk_jvmti_resumeSync 0000000180007a0c     libsuspendthrd003.obj
 0002:00002a0c       $unwind$nsk_jvmti_setFailStatus 0000000180007a0c     libsuspendthrd003.obj
 0002:00002a0c       $unwind$__scrt_initialize_default_local_stdio_options 0000000180007a0c     MSVCRT:default_local_stdio_options.obj
 0002:00002a0c       $unwind$?dllmain_crt_dispatch@@YAHQEAUHINSTANCE__@@KQEAX@Z 0000000180007a0c     MSVCRT:dll_dllmain.obj
 0002:00002a0c       $unwind$DllMain            0000000180007a0c     MSVCRT:dll_dllmain_stub.obj
 0002:00002a0c       $unwind$__GSHandlerCheck   0000000180007a0c     MSVCRT:gshandler.obj
 0002:00002a0c       $unwind$?__scrt_uninitialize_thread_safe_statics@@YAXXZ 0000000180007a0c     MSVCRT:thread_safe_statics.obj
 0002:00002a0c       $unwind$__scrt_acquire_startup_lock 0000000180007a0c     MSVCRT:utility.obj
 0002:00002a0c       $unwind$__scrt_dllmain_after_initialize_c 0000000180007a0c     MSVCRT:utility.obj
 0002:00002a0c       $unwind$__scrt_dllmain_before_initialize_c 0000000180007a0c     MSVCRT:utility.obj
 0002:00002a0c       $unwind$__scrt_dllmain_crt_thread_attach 0000000180007a0c     MSVCRT:utility.obj
 0002:00002a0c       $unwind$__scrt_dllmain_crt_thread_detach 0000000180007a0c     MSVCRT:utility.obj
 0002:00002a0c       $unwind$__scrt_dllmain_uninitialize_c 0000000180007a0c     MSVCRT:utility.obj
 0002:00002a0c       $unwind$__scrt_dllmain_uninitialize_critical 0000000180007a0c     MSVCRT:utility.obj
 0002:00002a0c       $unwind$atexit             0000000180007a0c     MSVCRT:utility.obj
 0002:00002a14       $unwind$nsk_jvmti_threadByName 0000000180007a14     libsuspendthrd003.obj
 0002:00002a2c       $unwind$nsk_jvmti_lverify  0000000180007a2c     libsuspendthrd003.obj
 0002:00002a40       $unwind$exitOnError        0000000180007a40     libsuspendthrd003.obj
 0002:00002a50       $unwind$check_option       0000000180007a50     libsuspendthrd003.obj
 0002:00002a50       $unwind$_DllMainCRTStartup 0000000180007a50     MSVCRT:dll_dllmain.obj
 0002:00002a60       $unwind$Java_nsk_share_jvmti_ArgumentHandler_getAgentOptionsString 0000000180007a60     libsuspendthrd003.obj
 0002:00002a74       $unwind$Java_nsk_jvmti_unit_FollowReferences_FollowRefObjects_getTag 0000000180007a74     libsuspendthrd003.obj
 0002:00002a74       $unwind$Java_nsk_share_jvmti_DebugeeClass_checkStatus 0000000180007a74     libsuspendthrd003.obj
 0002:00002a74       $unwind$agentThreadWrapper 0000000180007a74     libsuspendthrd003.obj
 0002:00002a84       $unwind$agentProc          0000000180007a84     libsuspendthrd003.obj
 0002:00002a84       $unwind$startAgentThreadWrapper 0000000180007a84     libsuspendthrd003.obj
 0002:00002aa0       $unwind$syncDebuggeeStatus 0000000180007aa0     libsuspendthrd003.obj
 0002:00002aa0       $unwind$__scrt_dllmain_exception_filter 0000000180007aa0     MSVCRT:utility.obj
 0002:00002ab4       $unwind$Java_nsk_share_jvmti_DebugeeClass_resetAgentData 0000000180007ab4     libsuspendthrd003.obj
 0002:00002abc       $unwind$MA_checkStatus     0000000180007abc     libsuspendthrd003.obj
 0002:00002ad0       $unwind$Java_nsk_jvmti_unit_FollowReferences_FollowRefObjects_setTag 0000000180007ad0     libsuspendthrd003.obj
 0002:00002ae8       $unwind$Java_nsk_jvmti_unit_FollowReferences_FollowRefObjects_addRefToVerify 0000000180007ae8     libsuspendthrd003.obj
 0002:00002b04       $unwind$Agent_Initialize   0000000180007b04     libsuspendthrd003.obj
 0002:00002b20       $unwind$capture_previous_context 0000000180007b20     MSVCRT:gs_report.obj
 0002:00002b2c       $unwind$__GSHandlerCheckCommon 0000000180007b2c     MSVCRT:gshandler.obj
 0002:00002b38       $xdatasym                  0000000180007b38     MSVCRT:amdsecgs.obj
 0002:00002b3c       $unwind$?dllmain_crt_process_attach@@YAHQEAUHINSTANCE__@@QEAX@Z 0000000180007b3c     MSVCRT:dll_dllmain.obj
 0002:00002b78       $unwind$?fin$0@?0??dllmain_crt_process_attach@@YAHQEAUHINSTANCE__@@QEAX@Z@4HA 0000000180007b78     MSVCRT:dll_dllmain.obj
 0002:00002b78       $unwind$?fin$0@?0??dllmain_crt_process_detach@@YAH_N@Z@4HA 0000000180007b78     MSVCRT:dll_dllmain.obj
 0002:00002b78       $unwind$?fin$1@?0??dllmain_crt_process_detach@@YAH_N@Z@4HA 0000000180007b78     MSVCRT:dll_dllmain.obj
 0002:00002b80       $unwind$?dllmain_crt_process_detach@@YAH_N@Z 0000000180007b80     MSVCRT:dll_dllmain.obj
 0002:00002bd4       $unwind$?dllmain_dispatch@@YAHQEAUHINSTANCE__@@KQEAX@Z 0000000180007bd4     MSVCRT:dll_dllmain.obj
 0002:00002bfc       $unwind$?filt$0@?0??dllmain_dispatch@@YAHQEAUHINSTANCE__@@KQEAX@Z@4HA 0000000180007bfc     MSVCRT:dll_dllmain.obj
 0002:00002c04       $unwind$__scrt_is_nonwritable_in_current_image 0000000180007c04     MSVCRT:utility.obj
 0002:00002c24       $unwind$__scrt_is_nonwritable_in_current_image$filt$0 0000000180007c24     MSVCRT:utility.obj
 0002:00002c2c       $unwind$__scrt_fastfail    0000000180007c2c     MSVCRT:utility_desktop.obj
 0002:00002c3c       $unwind$__security_init_cookie 0000000180007c3c     MSVCRT:gs_support.obj
 0002:00002c48       $unwind$__isa_available_init 0000000180007c48     MSVCRT:cpu_disp.obj
 0002:00002c58       $xdatasym                  0000000180007c58     MSVCRT:guard_dispatch.obj
 0002:00002c60       $xdatasym                  0000000180007c60     MSVCRT:guard_xfg_dispatch.obj
 0002:00002c70       .edata                     0000000180007c70     suspendthrd003.exp
 0002:00002c98       rgpv                       0000000180007c98     suspendthrd003.exp
 0002:00002cd0       rgszName                   0000000180007cd0     suspendthrd003.exp
 0002:00002d08       rgwOrd                     0000000180007d08     suspendthrd003.exp
 0002:00002d24       szName                     0000000180007d24     suspendthrd003.exp
 0002:00002d37       $N00001                    0000000180007d37     suspendthrd003.exp
 0002:00002d46       $N00002                    0000000180007d46     suspendthrd003.exp
 0002:00002d53       $N00003                    0000000180007d53     suspendthrd003.exp
 0002:00002d98       $N00004                    0000000180007d98     suspendthrd003.exp
 0002:00002dd5       $N00005                    0000000180007dd5     suspendthrd003.exp
 0002:00002e1d       $N00006                    0000000180007e1d     suspendthrd003.exp
 0002:00002e5d       $N00007                    0000000180007e5d     suspendthrd003.exp
 0002:00002e9a       $N00008                    0000000180007e9a     suspendthrd003.exp
 0002:00002ed5       $N00009                    0000000180007ed5     suspendthrd003.exp
 0002:00002f03       $N00010                    0000000180007f03     suspendthrd003.exp
 0002:00002f34       $N00011                    0000000180007f34     suspendthrd003.exp
 0002:00002f63       $N00012                    0000000180007f63     suspendthrd003.exp
 0002:00002f92       $N00013                    0000000180007f92     suspendthrd003.exp
 0002:00002fc7       $N00014                    0000000180007fc7     suspendthrd003.exp
 0002:00003432       .idata$6                   0000000180008432     kernel32:KERNEL32.dll
 0002:00003496       .idata$6                   0000000180008496     vcruntime:VCRUNTIME140.dll
 0002:00003632       .idata$6                   0000000180008632     ucrt:api-ms-win-crt-heap-l1-1-0.dll
 0002:00003652       .idata$6                   0000000180008652     ucrt:api-ms-win-crt-runtime-l1-1-0.dll
 0002:00003674       .idata$6                   0000000180008674     ucrt:api-ms-win-crt-convert-l1-1-0.dll
 0002:00003696       .idata$6                   0000000180008696     ucrt:api-ms-win-crt-stdio-l1-1-0.dll
 0002:000036b6       .idata$6                   00000001800086b6     ucrt:api-ms-win-crt-string-l1-1-0.dll
 0003:00000000       ?codeAttributeName@@3PEBDEB 0000000180009000     libsuspendthrd003.obj
 0003:00000008       ?lineNumberAttributeName@@3PEBDEB 0000000180009008     libsuspendthrd003.obj
 0003:00000010       ?localVarAttributeName@@3PEBDEB 0000000180009010     libsuspendthrd003.obj
 0003:00000018       ?localVarTypeAttributeName@@3PEBDEB 0000000180009018     libsuspendthrd003.obj
 0003:00000020       ?stackMapAttributeName@@3PEBDEB 0000000180009020     libsuspendthrd003.obj
 0003:00000028       ?callBytes@@3PAEA          0000000180009028     libsuspendthrd003.obj
 0003:0000002c       ?allocBytes@@3PAEA         000000018000902c     libsuspendthrd003.obj
 0003:0001aad4       redefineAttempted          0000000180023ad4     libsuspendthrd003.obj
 0003:0001aad8       nsk_context                0000000180023ad8     libsuspendthrd003.obj
 0003:0001aae4       redefineSucceed            0000000180023ae4     libsuspendthrd003.obj
 0003:0001aae8       agentFailed                0000000180023ae8     libsuspendthrd003.obj
 0003:0001aaec       currentAgentStatus         0000000180023aec     libsuspendthrd003.obj
 0003:0001aaf0       context                    0000000180023af0     libsuspendthrd003.obj
 0003:0001aba8       agentThread                0000000180023ba8     libsuspendthrd003.obj
 0003:0001abb0       agentThreadProc            0000000180023bb0     libsuspendthrd003.obj
 0003:0001abb8       agentThreadArg             0000000180023bb8     libsuspendthrd003.obj
 0003:0001abc0       agent_data                 0000000180023bc0     libsuspendthrd003.obj
 0003:0001abd0       jvmti_env                  0000000180023bd0     libsuspendthrd003.obj
 0003:0001abd8       jvm                        0000000180023bd8     libsuspendthrd003.obj
 0003:0001abe0       jni_env                    0000000180023be0     libsuspendthrd003.obj
 0003:0001abe8       checkStatus_func           0000000180023be8     libsuspendthrd003.obj
 0003:0001abf0       ?codeAttributeIndex@@3GA   0000000180023bf0     libsuspendthrd003.obj
 0003:0001abf4       ?lineNumberAttributeIndex@@3GA 0000000180023bf4     libsuspendthrd003.obj
 0003:0001abf8       ?localVarAttributeIndex@@3GA 0000000180023bf8     libsuspendthrd003.obj
 0003:0001abfc       ?localVarTypeAttributeIndex@@3GA 0000000180023bfc     libsuspendthrd003.obj
 0003:0001ac00       ?stackMapAttributeIndex@@3GA 0000000180023c00     libsuspendthrd003.obj
 0003:0001ac04       ?stackFrameOffset@@3GA     0000000180023c04     libsuspendthrd003.obj
 0003:0001ac08       ?mode@@3HA                 0000000180023c08     libsuspendthrd003.obj
 0003:0001ac0c       ?constantPoolSize@@3GA     0000000180023c0c     libsuspendthrd003.obj
 0003:0001ac10       ?orig@@3PEBEEB             0000000180023c10     libsuspendthrd003.obj
 0003:0001ac18       ?gen@@3PEAEEA              0000000180023c18     libsuspendthrd003.obj
 0003:0001ac20       ?inputPos@@3PEAEEA         0000000180023c20     libsuspendthrd003.obj
 0003:0001ac28       ?endPos@@3PEBEEB           0000000180023c28     libsuspendthrd003.obj
 0003:0001ac30       ?genPos@@3PEAEEA           0000000180023c30     libsuspendthrd003.obj
 0003:0001ac38       ?markPos@@3PEAEEA          0000000180023c38     libsuspendthrd003.obj
 0003:0001ac40       ?constantPool@@3PEAPEADEA  0000000180023c40     libsuspendthrd003.obj
 0003:0001ac48       ?constantPoolCount@@3GA    0000000180023c48     libsuspendthrd003.obj
 0003:0001ac4c       ?zeroBytes@@3PAEA          0000000180023c4c     libsuspendthrd003.obj
 0003:0001ac50       ?codeLength@@3IA           0000000180023c50     libsuspendthrd003.obj
 0003:0001ac58       ?map@@3PEAIEA              0000000180023c58     libsuspendthrd003.obj
 0003:0001ac60       ?widening@@3PEACEA         0000000180023c60     libsuspendthrd003.obj
 0003:0001ac68       timeout                    0000000180023c68     libsuspendthrd003.obj
 0003:0001ac80       ?str@?1??TranslateState@@YAPEBDH@Z@4PADA 0000000180023c80     libsuspendthrd003.obj
 0003:0001adb0       GS_ExceptionRecord         0000000180023db0     MSVCRT:gs_report.obj
 0003:0001ae50       GS_ContextRecord           0000000180023e50     MSVCRT:gs_report.obj
 0003:0001b320       ?g_tss_cv@@3U_RTL_CONDITION_VARIABLE@@A 0000000180024320     MSVCRT:thread_safe_statics.obj
 0003:0001b328       ?g_tss_event@@3PEAXEA      0000000180024328     MSVCRT:thread_safe_statics.obj
 0003:0001b330       ?g_tss_mutex@@3U_RTL_CRITICAL_SECTION@@A 0000000180024330     MSVCRT:thread_safe_statics.obj
 0003:0001b358       ?g_sleep_condition_variable_cs@@3P6AHPEAU_RTL_CONDITION_VARIABLE@@PEAU_RTL_CRITICAL_SECTION@@K@ZEA 0000000180024358     MSVCRT:thread_safe_statics.obj
 0003:0001b360       ?g_wake_all_condition_variable@@3P6AXPEAU_RTL_CONDITION_VARIABLE@@@ZEA 0000000180024360     MSVCRT:thread_safe_statics.obj
 0003:0001b36c       ?__proc_attached@@3HA      000000018002436c     MSVCRT:dll_dllmain.obj
 0003:0001b380       ?is_initialized_as_dll@@3_NA 0000000180024380     MSVCRT:utility.obj
 0003:0001b381       ?module_local_atexit_table_initialized@@3_NA 0000000180024381     MSVCRT:utility.obj
 0003:0001b388       ?module_local_atexit_table@@3U_onexit_table_t@@A 0000000180024388     MSVCRT:utility.obj
 0003:0001b3a0       ?module_local_at_quick_exit_table@@3U_onexit_table_t@@A 00000001800243a0     MSVCRT:utility.obj
